:100000000C9436030C9489030C9489030C94890393
:100010000C9489030C9489030C9489030C94890330
:100020000C9489030C9489030C941E240C9489036A
:100030000C94D5310C9489030C9489030C94890396
:100040000C9489030C9489030C9489030C94890300
:100050000C9489030C94FB0D0C9489030C94890374
:100060000C9489030C9489030C9489030C948903E0
:100070000C9489030C9489030C9489030C948903D0
:100080000C9489030C9489030C9489030C948903C0
:100090000C9489030C9489030C9489030C948903B0
:1000A0000C9489030C9489030C9489036C22932289
:1000B0008B2393228B23DF2202238B235923682354
:1000C0006F286F28A728A728022B022B022B022BB0
:1000D0002229022BFE28FE28BC2A022BD12AEF2A35
:1000E000000000000405060708090A0B0C0D0E0F9E
:1000F000101112131415161718191A1B1C1D1E1F88
:10010000202122232425262728292A2B2C2D2E2F77
:10011000303132333435363738393A3B3C3D3E3F67
:10012000404142434445464748494A4B4C4D4E4F57
:10013000505152535455565758595A5B5C5D5E5F47
:10014000606162636465A56768696A6B6C6D6E6FF8
:10015000707172737475767778797A7B7C7D7EA8FE
:10016000A9AA00000085008788898A8B000000000A
:10017000909100000000000000000000000000005E
:10018000000000000000000000000000000000006F
:10019000000000000000000000000000000000005F
:1001A000000000000000000000000000000000004F
:1001B000000000000000000000000000000000003F
:1001C000E0E1E2E3E4E5E6E7000000000000000013
:1001D000000000000000000000000000000000001F
:1001E00073706565643A2025730A007573625F73E6
:1001F000746174653A20253032580A00686F737450
:100200002E5461736B3A2025640A000D0A00200009
:100210000D0A0028686964626F6F742E682920498E
:100220006E746572666163653A000D0A002868693C
:1002300064626F6F742E682920537472616E6765F3
:10024000207265616420636F756E743A20000D0A38
:100250000028686964626F6F742E682920506F6C83
:100260006C3A000D0A0028686964626F6F742E682A
:1002700029206570496E666F5B6570496E746572A2
:1002800072757074496E496E646578202B20695DC3
:100290002E6D6178506B7453697A653D000D0A00CC
:1002A00028686964626F6F742E6829206570496ED2
:1002B000666F5B6570496E74657272757074496EB5
:1002C000496E646578202B20695D2E6570416464F9
:1002D000723D000D0A0028686964626F6F742E68B1
:1002E0002920693D0053657450726F746F3A004263
:1002F0004D20636F6E666967757265640D0A000D47
:100300000A0052504950452072636F64653A000DEF
:100310000A005345545F49444C452072636F64653D
:100320003A000D0A0050524F544F434F4C20534552
:1003300054204849445F424F4F542072636F6465B4
:100340003A000D0A000D0A496E74657266616365B4
:100350003A000D0A00624E756D49666163653A00A8
:100360000D0A006249666163654E756D3A000D0ABB
:1003700000436E663A000D0A00624E756D45503AB4
:10038000004849445F50524F544F434F4C5F4B45D8
:1003900059424F4152440D0A000D0A004E433A00A3
:1003A0000D0A00416464723A000D0A0073657441DD
:1003B0006464723A006570696E666F0D0A00424DA2
:1003C00020496E69740D0A00526F6C6C6F7665720D
:1003D000206572726F723A2069676E6F7265640D84
:1003E0000A000D0A00202530325800696E707574BD
:1003F0002025643A0054332000543220000D0A00B6
:10040000285553423A3A496E5472616E736665726A
:1004100029206570207265717565737465642000AC
:100420000D0A00285553423A3A496E5472616E7370
:1004300066657229206164647220726571756573E6
:1004400074656420000D0A00285553423A3A496EFB
:100450005472616E736665722920536574416464D9
:1004600072657373204661696C656420000D0A0033
:10047000637253543A000D0A0063724F55543A00A8
:10048000436F2000543120000D0A006372494E3A38
:1004900000436920000D0A00637253553A000D0AAB
:1004A00000637253413A002E2E2E4641494C0D0AEC
:1004B0000042756666657220706F696E74657220A1
:1004C0006973204E554C4C210D0A000D0A000D0A8F
:1004D000736574436F6E6620000D0A67657444652A
:1004E00076446573637220000A4B6579626F6172AE
:1004F000642073746172742E0A000A55534220639B
:100500006F6E666967757265642E0A000A0A544D3B
:100510004B3A32623734323033622B2F4C554641DE
:100520000A0A003C03550053004200200074006F8B
:1005300000200055005300420020006B0065007948
:100540000062006F00610072006400200063006FB1
:10055000006E007600650072007400650072000095
:10056000000E0374002E006D002E006B002E0000A4
:10057000000403090409024200020100A032090438
:1005800000000103010100092111010001224000C6
:100590000705810308000A090401000203000000A6
:1005A0000921110100012222000705820320000118
:1005B000070502032000011201100100000008EDF0
:1005C000FE5B001408010200010631FF0974A1015D
:1005D0000975150026FF009520750881020976151A
:1005E0000026FF00952075089102C005010906A1AB
:1005F00001050719E029E715002501950875018116
:1006000002950175088101050819012905950575EF
:100610000191029501750391010507190029FF1544
:100620000026FF00950675088100C0636F6E737524
:100630006D65723A20253034580A007379737465F9
:100640006D3A20253034580A000A002530325820EF
:10065000006B6579626F6172643A20004C45443AE0
:1006600020253032580A0000AB0C660D11241FBE45
:10067000CFEFDAE0DEBFCDBF04B603FE28C0809125
:10068000B5059091B605A091B705B091B805873032
:10069000904BA740B04BD9F41092B5051092B60517
:1006A0001092B7051092B80514BE0FB6F894A8952D
:1006B00080916000886180936000109260000FBE9E
:1006C0001092010810920008E0E0F8E3099511E0AB
:1006D000A0E0B1E0ECECF8E602C005900D92A6387F
:1006E000B107D9F725E0A6E8B1E001C01D92A53B0E
:1006F000B207E1F713E0C6E3D3E004C02197FE019F
:100700000E945E34C433D107C9F70E947E1F0C9447
:1007100064340C940000FF93EF93E0918601F09114
:100720008701309709F00995EF91FF910895FC0139
:100730008591803011F0EFDFFBCF0895FF27E0E2D5
:1007400030E247FF0CC0419597FF09C0EDE260958C
:10075000709580959095611D711D811D911D27FFDC
:1007600002C0219530E350E2AA27660F771F881F49
:10077000991FAA1FA41710F0A41B63955A95A9F7F7
:10078000AA3008F0A95FA05DAF93F39561157105DC
:100790008105910541F7ED3211F4EF93F395F217CE
:1007A00018F43F93F395FBCF8F91B5DFFA95E1F7FE
:1007B0000895E991F9918591803021F0853219F001
:1007C000AADFF9CF089520E0E89455915532C1F39E
:1007D000503311F4689455915A3348F4505390F3C0
:1007E000220F022E220F220F200D250FF4CF0EF420
:1007F000219589919991533619F3533729F153353E
:1008000059F1BC0188279927E8945C3621F4899135
:10081000999168945591543639F446EF7EF077FFFC
:100820000DC08FEF9FEF0AC055374AE039F05835B9
:1008300040E121F0523642E009F00895FF93EF9332
:100840007DDFEF91FF91B7CFFF93EF93FC01819193
:100850008030B9F360DFFBCFFF93EF9368DFF1CF18
:10086000DF93CF93CDB7DEB72596A3DFCF91DF918E
:10087000089580E00895089580E0089581E0089546
:10088000CF93DF93CDB7DEB728970FB6F894DEBFCE
:100890000FBECDBFE22F29833A834B835C836D83E8
:1008A0007E838F8398878091C402E82BE093C402F3
:1008B000FE013396AE01475F5F4F2191243088F0EF
:1008C000A6ECB2E080E090E03D91311106C0DC0181
:1008D000AC53BD4F12962C9304C0019686309105FF
:1008E00099F7E417F50749F728960FB6F894DEBF95
:1008F0000FBECDBFDF91CF910895860F911D860F5A
:10090000911DFC015687458781E00895FC01878988
:100910000895CF93DF93EC018C819D81DC01ED91F3
:10092000FC910480F581E02D6E8109951F86188A5F
:1009300081E08A8B1E821B8A1C8A1D8A1E8A1F8A5E
:1009400080E0DF91CF910895FC018681089581E0D8
:10095000633009F080E0089581E0613009F080E0C3
:100960000895860F911D860F911DFC018585968542
:100970000895EF92FF92CF93DF93DC01E701529647
:100980008C915297823049F11F966C931F97509625
:100990004C9350979B8193709330F9F49A8197FF11
:1009A0001CC09E8158962C915897291718F4589678
:1009B0009C935897E82FF0E09F01220F331FE20F1E
:1009C000F31FEA0FFB1F9A819F7097839C8190878A
:1009D00094E091878F5F52968C93DF91CF91FF9037
:1009E000EF900895EF92FF920F9302970E94B9043F
:1009F0000F91FF90EF90089508953F924F925F926C
:100A00006F927F928F929F92AF92BF92CF92DF921E
:100A1000EF92FF920F931F93CF93DF9300D000D0FC
:100A2000CDB7DEB76C017C836B835A8349834C015D
:100A300080E1880E911C5601A7E0AA0EB11C11E0BE
:100A400084E0482E3601B2E16B0E711C93E0392E22
:100A500022E0522E8B819C81892B09F4FBC0F60188
:100A600080A1823059F128F4882341F0813071F05F
:100A7000F1CF833039F18430C1F1ECCF54828581DC
:100A80009681908787835286518610A3AE014D5F71
:100A90005F4FBE016F5F7F4FC5010E94C01C88235E
:100AA00009F4D8C0D6011596ED91FC911697808176
:100AB00091968C939197818192968C93F601768290
:100AC000658230A2D60192968C919297843011F46F
:100AD00093961C92F60181A18250848325813681F0
:100AE000308727838287818740A2D60192968C9196
:100AF0008430B1F0853009F442C0823009F06EC014
:100B0000AE014D5F5F4FBE016F5F7F4FC5010E9419
:100B1000C01C882309F49EC0F601858984A392C075
:100B2000AE014D5F5F4FBE016F5F7F4FC5010E94F9
:100B3000C01C882309F48EC0D60155968C91559718
:100B4000833009F07FC056968C915697813009F01A
:100B500079C098969C91989757968C91992321F0FB
:100B6000882309F46FC003C0813009F06BC0F6011F
:100B700013A3928996A3938997A385A363C0AE011B
:100B80004D5F5F4FBE016F5F7F4FC5010E94C01C6C
:100B9000882309F45FC0D60193968C91939788239C
:100BA00009F450C012968D919C911397009709F407
:100BB00049C0DC01ED91FC910190F081E02D7401C0
:100BC000D60195960C91959797962C919797969616
:100BD0004C91969794966C91099534C0F601858551
:100BE000882319F0813039F028C081A190E0029764
:100BF0009787868715872B813C8189819A81782FF9
:100C0000692FF601468557854115510581F00196FA
:100C10002115310529F41C821B8279836A830DC05A
:100C2000415051095787468721503109E8CF3C830D
:100C30002B839A838983F6011586F601868597852D
:100C4000892B41F4D60116969C928E921597909618
:100C50001C9200CF0F900F900F900F90DF91CF91CB
:100C60001F910F91FF90EF90DF90CF90BF90AF90CA
:100C70009F908F907F906F905F904F903F900895DE
:100C8000CF93DF936091E2017091E301E0918F01D6
:100C9000F09190014091D6015091D7012091CA0165
:100CA0003091CB018091BE019091BF016E177F07FB
:100CB000B1F4E0918D01F0918E014E175F0779F448
:100CC000E0918B01F0918C012E173F0741F4E091E8
:100CD0008901F0918A018E179F0709F463C0709310
:100CE000900160938F0150938E0140938D0130935A
:100CF0008C0120938B0190938A0180938901E4EC0D
:100D0000F2E088E0DF011D928A95E9F72091DA018F
:100D10003091DB014091DC015091DD016091DE01F9
:100D20007091DF018091E0019091E1010E94400407
:100D30002091CE013091CF014091D0015091D1014D
:100D40006091D2017091D3018091D4019091D5012D
:100D50000E9440042091C2013091C3014091C4011E
:100D60005091C5016091C6017091C7018091C80181
:100D70009091C9010E9440042091B6013091B701C1
:100D80004091B8015091B9016091BA017091BB01D5
:100D90008091BC019091BD010E94400481E080934C
:100DA000C30202C01092C3020E94D40DEC018CE475
:100DB00092E00E940C17CE010E94EC0D8536910541
:100DC00060F09F938F938CEF91E09F938F930E949D
:100DD00030040F900F900F900F908CE492E00E94DF
:100DE0002C0F90918801891779F18CE492E00E9490
:100DF0002C0F809388011F928F938BEE91E09F932D
:100E00008F930E9430040F900F900F900F9080915D
:100E100088018039C9F480919101823019F08AE10A
:100E200091E002C085E191E09F938F9380EE91E085
:100E30009F938F930E9430040E940C250E94782675
:100E40000F900F900F900F9081E0DF91CF91089558
:100E5000482F80E1489F90011124205E31092830FD
:100E6000310538F49091C402992319F0892F90E04C
:100E700002C080E090E0E6ECF2E061E070E02191F9
:100E8000243070F0322F32953F70431309C02F7019
:100E9000DB0102C0AA0FBB1F2A95E2F78A2B9B2B0E
:100EA000B2E0EC3CFB0759F708950895CF92DF922A
:100EB000EF92FF920F93CF93DF931F92CDB7DEB7E0
:100EC000898380914902882371F0CE0101966C01DB
:100ED000EE24E394F12C00E022E040E060E082E3C5
:100EE00092E00E94601880912F02882371F0CE0159
:100EF00001966C01EE24E394F12C00E022E040E046
:100F000060E088E192E00E946018809115028823D9
:100F100071F0CE0101966C01EE24E394F12C00E017
:100F200022E040E060E08EEF91E00E946018809146
:100F3000FB01882371F0CE0101966C01EE24E3944D
:100F4000F12C00E022E040E060E084EE91E00E94BD
:100F500060180F90DF91CF910F91FF90EF90DF908D
:100F6000CF9008950E9493318091AA05882331F093
:100F70000E94BC31882321F00C949A200C944006E6
:100F80000895FC01758364838EE291E091838083F0
:100F90008CE491E093838283138A148A158A168ADB
:100FA000178A418F178288E080878CE381871286B9
:100FB000138684E0848781E0828B118A17861686E7
:100FC000158661157105B1F0DB01AA5ABF4F80E0AB
:100FD00090E02D913D91232B49F48B96880F991F1A
:100FE000DB01A80FB91FED93FC93089501968031A2
:100FF000910579F708952E9A08952E988EBD0DB417
:1010000007FEFDCF1EBC0DB407FEFDCF0E94FB07FF
:101010008EB508952E9882608EBD0DB407FEFDCF6B
:101020006EBD0DB407FEFDCF0C94FB0788EF0E9448
:10103000FD07807C803411F118F4882371F1089544
:10104000803819F0803C39F1089588ED0E94FD0741
:101050009091910181FD08C0923029F161EC88EDF9
:101060000E940A0882E007C09330E9F063EC88ED43
:101070000E940A0883E080939101089588ED0E9400
:10108000FD079091910181FD03C0933079F7089598
:10109000923021F7089581E0EECF61ED88ED0E9456
:1010A0000A081092910108950F931F93CF93DF9335
:1010B0008C01269A0E94FB07219A229A2398209A53
:1010C00080E58CBD81E08DBD259868E188E80E94AF
:1010D0000A0860E288E70E940A0860E088E70E9448
:1010E0000A08C0E0D0E088E60E94FD07219680FD56
:1010F00006C0CF3F8FEFD807B1F78FEF1DC061EC6F
:1011000088ED0E940A0860E280ED0E940A0864E00F
:1011100088EE0E940A0888EE0E94FD0782FFFBCF3E
:10112000C8010E94160860E288EC0E940A0861E08B
:1011300080E80E940A0880E0DF91CF911F910F9113
:1011400008958091A60581608093A6058CE492E0C5
:101150000E94540888ED91E09093400280933F02F2
:101160008CEC91E0909326028093250280EC91E034
:1011700090930C0280930B0284EB91E09093F20128
:101180008093F10108950F931F93CF93C82F8B0184
:10119000282F30E084E0359527958A95E1F780E3A4
:1011A000820F8A3310F087E3820FB8010E94FB1C84
:1011B000CF7080E38C0F8A3310F087E38C0FB80177
:1011C000CF911F910F910C94FB1C2F923F924F9245
:1011D0005F926F927F928F929F92AF92BF92CF92C7
:1011E000DF92EF92FF920F931F93CF93DF93CDB7D0
:1011F000DEB7EB970FB6F894DEBF0FBECDBF7C0114
:10120000362E242E422EDC011496AD90BC901597FC
:1012100060E870E08EEB93E00E94081DF7015680B5
:10122000511012C2108ED501ED91FC910190F08108
:10123000E02D60E0C50109956C01009719F446EDB9
:10124000542E07C2FC01808091808114910449F4DE
:1012500060E870E085EB93E00E94081D37ED532EA7
:10126000F8C13701F7E06F0E711CDC0111967C921A
:101270006E9214964C928E01065D1F4F28E030E06E
:1012800040E060E0F701848195810E945914182F95
:101290008111C3C11AA5D6018D929C92D501ED9101
:1012A000FC910280F381E02D222D40E0632DC501E9
:1012B0000995F7018683882309F4C9C199A9908704
:1012C000282F40E060E0848195810E940415982ECB
:1012D000882319F1D60114961C92D501ED91FC9149
:1012E0000480F581E02DD70116966C91C501099512
:1012F000F701168260E870E08CEA93E00E94081D16
:1013000060E870E0892D0E94C30860E870E089EA17
:1013100093E00E94081D592C9CC160E870E083EAAC
:1013200093E00E94081D60E870E0D70116968C914A
:101330000E94C30860E870E080EA93E00E94081D04
:10134000F6011482D501ED91FC910190F081E02D20
:10135000D70116966C91C5010995009709F46FCFD6
:10136000133108F012E1FC014482930141E0D701FE
:1013700016966C91169714968D919C9115970E94D4
:101380004C0F111126C03BAC60E870E08CE993E093
:101390000E94081D60E870E0832D0E94C30860E889
:1013A00070E089E993E00E94081D60E870E081E840
:1013B00093E00E94081D412C22E2822E21E0922E11
:1013C0005701B2E0AB0EB11C6E01E1E1CE0ED11CB3
:1013D00039C0212F30E08E01065D1F4F40E0D7015C
:1013E00016966C91169714968D919C9115970E9464
:1013F0005914182F811114C1C6CF9A828982BC82D8
:10140000AB821D821A861B861E86188A1F8619A229
:101410001AA21BA219A6DF82CE82D986C886DD86D3
:10142000CC868E010F5F1F4F242D40E0F7016681AF
:10143000848195810E94A714D70152968C918230A5
:1014400019F043944310D9CF60E870E089E793E046
:101450000E94081D60E870E0F70182890E94C308BD
:1014600060E870E086E793E00E94081DD70152967D
:101470008C915297823009F0D9C0930142E01696C0
:101480006C91169714968D919C9115970E944C0F14
:1014900060E870E081E793E00E94081D60E870E07A
:1014A000F70187850E94C30860E870E08EE693E04C
:1014B0000E94081D68EE73E080E090E00E947D0DC0
:1014C000D7011F962C911F9740E016966C911697A6
:1014D00014968D919C9115970E947216182F811168
:1014E000A2C068EE73E080E090E00E947D0D60E8AD
:1014F00070E083E693E00E94081D60E870E0F70169
:1015000080890E94C30860E870E080E693E00E9452
:10151000081D60E870E085E593E00E94081D60E822
:1015200070E0D70151968C910E94C30860E870E08A
:1015300082E593E00E94081D60E870E085E493E096
:101540000E94081D60E870E080E00E94C30860E827
:1015500070E082E493E00E94081DF701418D60E095
:10156000C7010E94B718182F60E870E0811150C0C1
:1015700085E293E00E94081D60E870E080E00E9430
:10158000C30860E870E082E293E00E94081D20E05A
:1015900040E060E0C7010E948D18182F60E870E0FD
:1015A00082E193E00E94081D60E870E0812F0E94B4
:1015B000C30860E870E08FE093E00E94081D88E2B5
:1015C00091E09A838983AE014F5F5F4F60E070E0E6
:1015D000C7010E941D18182F60E870E082E093E0B8
:1015E0000E94081D60E870E0812F0E94C30860E837
:1015F00070E08FEF92E00E94081D60E870E08FEECF
:1016000092E00E94081D81E0D70157968C9321C07B
:1016100085EE92E00E94081D0AC0F6019182808248
:101620000E94261D04C00E942C1D01C011ED812FB7
:101630000E94321DD701ED91FC910480F581E02DCF
:10164000C7010995512E05C099ED592E02C084EDB0
:10165000582E852DEB960FB6F894DEBF0FBECDBF8A
:10166000DF91CF911F910F91FF90EF90DF90CF907E
:10167000BF90AF909F908F907F906F905F904F90B2
:101680003F902F900895EF92FF920F931F93CF9367
:10169000DF937C018B01CCE0D0E0C7010C2E02C0AF
:1016A000959587950A94E2F7982F9F7080E3890FAC
:1016B0008A3310F087E3890FB8010E94FB1C24973E
:1016C000CC3F8FEFD80749F7DF91CF911F910F9152
:1016D000FF90EF900895AF92BF92CF92DF92EF927A
:1016E000FF920F931F93CF93DF93CDB7DEB762972F
:1016F0000FB6F894DEBF0FBECDBFDC0157962C911C
:10170000222381F06C010E947B0DF601038914896C
:1017100025893689DC01CB01801B910BA20BB30B11
:10172000B7FF02C0F12C05C161E870E086ED92E0E0
:101730000E94081D61E870E080E090E00E94430B89
:1017400061E870E083ED92E00E94081D61E870E0BE
:1017500080EA92E00E94081D61E870E0D6011A96C6
:101760008C910E94C30861E870E08DE992E00E94CC
:10177000081D61E870E086E692E00E94081D61E8BD
:1017800070E0F60183850E94C30861E870E083E69B
:1017900092E00E94081DD6011B968C911B9790E049
:1017A0009A8B898BE12C8E010F5F1F4F9E012F5E5C
:1017B0003F4F1A964C911A9716966C91169714965D
:1017C0008D919C9115970E949716F82E882329F0E9
:1017D000F4E0FF1609F478C006C029893A8923305D
:1017E000310508F055C061E870E081E592E00E94A3
:1017F000081D61E870E08F2D0E94C30861E870E069
:101800008EE492E00E94081DF1105EC089899A89D9
:10181000892B09F459C060E870E08DE292E00E94E3
:10182000081DA988BA880CE010E0C501002E02C08E
:10183000969587950A94E2F7982F9F7080E3890F19
:101840008A3318F560E870E00E94FB1C045011090F
:101850000C3F8FEF180749F760E870E08AE292E0EA
:101860000E94081D60E870E083E192E00E94081D7C
:1018700060E870E080E090E00E94430B60E870E078
:1018800080E192E00E94081D2EC087E3890FDACF25
:10189000D6011D968D919C911E97009721F1DC0138
:1018A000ED91FC910190F081E02D8E010F5F1F4FB3
:1018B00040E0B601099517C0232B31F060E870E0D5
:1018C0008BE092E00E94081D0E947B0DF601208DA6
:1018D000DC01CB01820F911DA11DB11D838B948B67
:1018E000A58BB68B26C089899A89892B69F380914B
:1018F0000001909101018038910534F310E02989AD
:101900003A89812F90E082179307B0F6E1E0F0E08A
:10191000EC0FFD1FE80FF91F60E870E080810E9466
:10192000C30860E870E08EE092E00E94081D1F5F2F
:10193000E6CF8F2D62960FB6F894DEBF0FBECDBFF7
:10194000DF91CF911F910F91FF90EF90DF90CF909B
:10195000BF90AF9008958CE492E00E94FC0E40E0AE
:101960006CE472E082E392E00E94C10740E06CE424
:1019700072E088E192E00E94C10740E06CE472E00E
:101980008EEF91E00E94C10740E06CE472E084EECB
:1019900091E00E94C10782E591E09093D901809384
:1019A000D8019093CD018093CC019093C101809395
:1019B000C0019093B5018093B4016CE472E083EAB6
:1019C00091E00E94501B6CE472E082E991E00C947B
:1019D000501BAF92BF92CF92DF92EF92FF920F9384
:1019E0001F93CF93DF937C01CB01D22EDB01ED91CE
:1019F000FC910084F185E02D09951F928F938BEE69
:101A000093E09F938F930E943004E8015801AD0C3E
:101A1000B11C0F900F900F900F9085EEC82E83E0B1
:101A2000D82ECA15DB0561F089911F928F93DF9242
:101A3000CF920E9430040F900F900F900F90F1CF33
:101A400082EE93E09F938F930E9430040F900F904B
:101A5000F8018281813049F488EC93E09F938F9361
:101A60000E9430040F900F900FC0D701129688E0AB
:101A7000F80101900D928A95E1F70E947B0DD70144
:101A80001B967C936E931A97DF91CF911F910F91C4
:101A9000FF90EF90DF90CF90BF90AF90089580E0DF
:101AA00090E008958FEF9FEF089581E090E0089512
:101AB0000895862F0E94A81D81E090E00895FB0103
:101AC00080810E94A81D81E090E00895ECECF2E096
:101AD0001382128288EE93E0A0E0B0E084839583C5
:101AE000A683B78388E591E0918380838FEF9FEF92
:101AF0009587848708950C94E00D8F929F92AF9202
:101B0000BF92CF92DF92EF92FF920E943A334B0145
:101B10005C0120E030E04AE755E40E94F1336B01BC
:101B20007C0120E030E040E85FE30E94063387FD5F
:101B300024C020E03FEF4FE757E4C701B6010E9401
:101B4000EC331816ACF420E030E040E251E4C5017B
:101B5000B4010E94F1330E940B3320E931E061159A
:101B6000710581F0C9010197F1F761507109F7CF53
:101B7000C701B6010E940B3302C061E070E0CB01E7
:101B80000197F1F7FF90EF90DF90CF90BF90AF906B
:101B90009F908F90089582E084BD93E095BD9AEF69
:101BA00097BD80936E0008952FB7F89480911C0321
:101BB00090911D03A0911E03B0911F032FBF0895A4
:101BC0002FB7F89460911C0370911D0380911E0340
:101BD00090911F032FBF08959C014FB7F8948091F7
:101BE0001C0390911D03A0911E03B0911F034FBFD2
:101BF000821B930B089578941F920F920FB60F9249
:101C000011248F939F93AF93BF9380911C03909166
:101C10001D03A0911E03B0911F030196A11DB11DCC
:101C200080931C0390931D03A0931E03B0931F0386
:101C3000BF91AF919F918F910F900FBE0F901F900A
:101C40001895CF93DF93FC01862F8078A9F4283074
:101C500008F04DC0442321F09581973009F447C026
:101C6000EF01A1E0B0E09D85992341F01196259602
:101C7000A031B105C1F73BC080E039C061111CC083
:101C800085E08A9FE0018B9FD00D1124CE0FDF1FCE
:101C9000442331F081E4888785818F5F858302C08A
:101CA00081E0888725E02A9FC0012B9F900D112499
:101CB000E80FF91F80851BC06770660F660F660FFF
:101CC000442341F0606485818F5F85838770687FDE
:101CD000682B03C02770687B622B25E02A9FC00118
:101CE0002B9F900D1124E80FF91F6087862FDF913D
:101CF000CF910895611102C006960895FC0121E07C
:101D00003585631739F02F5F35962031C9F780E0AC
:101D100090E00895069635E0239F800D911D1124D3
:101D20000895DF92EF92FF920F931F93CF93DF936B
:101D3000EC01E62EF12C85E0689FB0011124FE0134
:101D4000E60FF71F8085182F177086FF17C001E078
:101D500085E0D82EFE01D09EE00DF11D1124808576
:101D600086958695869587701817F9F00F5F003174
:101D700089F78D81811302C011501D8385E08E9DEE
:101D8000F0018F9DF00D1124EC0FFD1F108681E0F6
:101D9000818712862296D783C683DF91CF911F91C8
:101DA0000F91FF90EF90DF900895602FCE010E9479
:101DB000910ED0CFFC01613499F49C01255B3F4F1B
:101DC00061E0AC014E5F5F4F1586668717865487CA
:101DD00043873596E217F307B9F7FC01158208959A
:101DE00021E03585631729F02F5F35962031C9F73B
:101DF0000895622F0C94910EFC018AE691E0918384
:101E000080831582108681E081871286CF01029639
:101E100097838683128228E023832CE32483DF01C7
:101E20009F01255B3F4F41E01D961C921D971E961A
:101E30004C931E971F961C921F971C969C938E93F3
:101E40001B971596A217B30779F7EA58FF4F108230
:101E500081E1809324030895809124030895CF9312
:101E6000C42F0E947A0E009789F0DC01ED91FC915D
:101E70001197309759F013969C9180E0891731F0B3
:101E800020812C1731F033968F5FF8CF80E090E0FF
:101E900001C0CF01CF9108950F931F93CF93DF938C
:101EA0002115310571F0E901042F162F0E947A0ED9
:101EB000FC01892B41F01283D183C083038380E02E
:101EC00003C088ED01C086EDDF91CF911F910F9186
:101ED0000895CF92DF92FF920F931F93CF93DF93DA
:101EE000662381F1F62E8C016C0186E5C80ED11CAB
:101EF000C0E0D0E0D6018D919D916D010097F1F089
:101F0000DC01ED91FC910084F185E02D0995F8123A
:101F100015C0AB96CC0FDD1FC00FD11F88819981F2
:101F2000DC01ED91FC910480F581E02DDF91CF91F2
:101F30001F910F91FF90DF90CF9009942196C031AF
:101F4000D105C1F680E0DF91CF911F910F91FF90F5
:101F5000DF90CF9008952E980895CF93C82F0E94B8
:101F6000AB0FCEBD0DB407FEFDCF1EBC0DB407FEFA
:101F7000FDCF0E94FB078EB5CF910895CF93DF93DD
:101F8000C82FD62F0E94AB0FC260CEBD0DB407FE86
:101F9000FDCFDEBD0DB407FEFDCFDF91CF910C94D8
:101FA000FB078F929F92AF92BF92CF92DF92EF92F8
:101FB000FF920F931F93CF93DF93EC01D62EC42E85
:101FC00059010E947A0E7C01009709F445C0FC017A
:101FD00080819181892B09F441C04C2D6D2DCE015A
:101FE0000E942F0FF501918380830097C9F1FC01B6
:101FF00082818695869590E08031910514F08FE07E
:1020000090E041E050E060E070E04A015B0104C014
:10201000880C991CAA1CBB1C8A95D2F7D501C40157
:102020000197F801918380836D2D80EE0E94BE0F91
:1020300088ED0E94AD0FF7019481992331F0CA58C1
:10204000DF4F68816260682B02C0682F697F88ED6E
:102050000E94BE0F80E005C086ED03C087ED01C081
:102060008BEDDF91CF911F910F91FF90EF90DF905B
:10207000CF90BF90AF909F908F9008958F929F9236
:10208000AF92BF92CF92DF92EF92FF920F931F9386
:10209000CF93DF93862E942E59010E947B0D6B0106
:1020A0007C0128E8C20E23E1D21EE11CF11C00E0F5
:1020B00010E0D0E0C0E098280E947B0DDC01CB014D
:1020C0008C199D09AE09BF09B7FF2DC0692D80EF9E
:1020D0000E94BE0F0E947B0DDC01CB018C199D0973
:1020E000AE09BF09B7FF09C088EC0E94AD0F87FF9A
:1020F000F1CF60E888EC0E94BE0F88EF0E94AD0F20
:10210000C82FCF70C43019F0CE3051F00CC00F5F23
:102110001F4FA114B10481F20A151B0569F603C013
:10212000DF5FD33049F68C2FDF91CF911F910F9154
:10213000FF90EF90DF90CF90BF90AF909F908F90E7
:1021400008959F92AF92BF92CF92DF92EF92FF924B
:102150000F931F93CF93DF937C01D42F122F902ED8
:1021600000E06C01C60ED11CC60ED11C86E5C80E5F
:10217000D11CA42EB12CABE2AA0EB11CAA0CBB1C24
:10218000AE0CBF1CF60180819181DC01ED91FC91C8
:102190000280F381E02D292D412F6D2F0995803E7E
:1021A000C9F4D1110BC061E088EE0E94BE0F66E653
:1021B00070E080E090E00E947D0D14C0F501808108
:1021C0009181DC01ED91FC910284F385E02D612F7A
:1021D000099508C08D3021F4033008F03FC014C0C9
:1021E00081113FC0F60180819181DC01ED91FC916C
:1021F0000190F081E02D292D412F6D2F0995C82FD9
:102200008D3051F4033050F464E670E080E090E0EB
:102210000E947D0D0F5FB6CF882311F1D1110BC045
:1022200061E088EE0E94BE0F66E670E080E090E01C
:102230000E947D0D11C0ED2FF0E0BB96EE0FFF1F49
:10224000EE0DFF1D80819181DC01ED91FC910284F6
:10225000F385E02D612F09958C2F03C08DE001C01F
:1022600080E0DF91CF911F910F91FF90EF90DF9071
:10227000CF90BF90AF909F9008950F931F93CF93EF
:10228000DF93182F062FEA010E94AB0F12601EBDCC
:10229000FE01802F882339F00DB407FEFDCF919108
:1022A0009EBD8150F7CFC00FD11D0DB407FEFDCFED
:1022B0000E94FB07CE01DF91CF911F910F910895EE
:1022C0002F923F924F925F926F927F928F929F9246
:1022D000AF92BF92CF92DF92EF92FF920F931F9334
:1022E000CF93DF9300D000D01F92CDB7DEB77B0134
:1022F0004A016901FB01F181F9838F2F81508034FC
:1023000008F074C00E947B0D2B013C0128E8420EAE
:1023100023E1521E611C711CF701828180FD02C005
:1023200060E401C060E888EE0E94BE0F312C998104
:10233000892F90E09A838983C114D10409F449C09C
:10234000E981FA81FD83EC83CE16DF0610F4DD828D
:10235000CC82FC81FB83A8016F2F80E10E943D119C
:102360006C8188E30E94BE0FF7016081606280EF9C
:102370000E94BE0F88EC0E94AD0F87FFFBCF60E884
:1023800088EC0E94BE0F88EF0E94AD0F8F70382E30
:10239000A12CB12C212C332009F45AC00E947B0DB2
:1023A000DC01CB0184199509A609B709B7FF50C014
:1023B0001FC02EE0321609F446C084E0381209C06E
:1023C000FFEFAF1ABF0A81149104D9F0A814B90421
:1023D000C1F488EF0E94AD0F85FB882780F9F701D3
:1023E000928180FB90F99283832D39C08AED37C0AA
:1023F000F6E03F12DECF60E870E085EF93E00E94E8
:10240000081D60E088E30E94BE0FF801608180E152
:102410000E94BE0F6B8188E30E94BE0FF7016081AE
:10242000606280EF0E94BE0F88EC0E94AD0F87FFB4
:10243000FBCF60E888EC0E94BE0F88EF0E94AD0FD2
:102440008F70382EA8CF239423E02212DACFC1CF89
:10245000EC81FD81CE1ADF0A0E0F1F1F6DCF0F908A
:102460000F900F900F900F90DF91CF911F910F91D0
:10247000FF90EF90DF90CF90BF90AF909F908F90A4
:102480007F906F905F904F903F902F9008952F9284
:102490003F924F925F926F927F928F929F92AF92F4
:1024A000BF92CF92DF92EF92FF920F931F93CF9341
:1024B000DF93CDB7DEB72A970FB6F894DEBF0FBE15
:1024C000CDBF9D838C836B015F834E835901EA826C
:1024D000F90180809180FB01F181FB83F901118278
:1024E0001082FB01828181FD02C060E101C060E2D7
:1024F00088EE0E94BE0FFA814F2E512C612C712C58
:1025000088862E813F81F601408160E08C819D812B
:102510000E943E108983863039F460E870E089EFCC
:1025200093E00E94081DEDCFF981F11163C088ECA2
:102530000E94AD0F82FF5CC080E30E94AD0F382E79
:1025400090E08816990608F43884F501808191811D
:102550009401281B390B3A87298737FF02C01A8656
:102560001986E32CF12C89859A85E816F90614F46E
:10257000FA86E98629840E94AB0F98E09EBD0DB4CF
:1025800007FEFDCFF801222041F01EBC2A940DB4B5
:1025900007FEFDCF8EB58193F6CFE985FA850E0F44
:1025A0001F1F0E94FB0764E088EC0E94BE0FF5012C
:1025B00080819181E80EF91EF182E082FB813F1655
:1025C00018F0E814F90458F088EF0E94AD0F8295D6
:1025D0008170F601928180FB91F992830BC0FA81A0
:1025E000FF2309F48ECFC301B2010E947D0D89CF74
:1025F00020EF298389812A960FB6F894DEBF0FBE9B
:10260000CDBFDF91CF911F910F91FF90EF90DF90A1
:10261000CF90BF90AF909F908F907F906F905F9082
:102620004F903F902F9008952F923F924F925F923C
:102630006F927F928F929F92AF92BF92CF92DF92D2
:10264000EF92FF920F931F93CF93DF93CDB7DEB737
:1026500061970FB6F894DEBF0FBECDBF3C01F42EDC
:10266000322E202EC98A65014EA05FA0A8A4B9A46D
:10267000188A1F861E861D868E01035F1F4F9E01CE
:10268000215F3F4F0E94D10F182F882381F060E80F
:1026900070E081EA94E00E94081D60E870E0812FFC
:1026A0000E94C30860E870E08EE994E029C0398296
:1026B0002A82EB82F989FC83DE82CD8298868F8222
:1026C000AE014F5F5F4F68E080E20E943D112D85B3
:1026D0003E854F2D60E1C3010E943E10182F8823D4
:1026E00091F060E870E088E994E00E94081D60E8DD
:1026F00070E0812F0E94C30860E870E085E994E0F3
:102700000E94081DB7C0832D8078382EA114B10413
:1027100009F46EC060E870E0332009F442C081E93A
:1027200094E00E94081DEF85F8898281826082838F
:102730006401C114D10409F459C09C2D8D2D4C1491
:102740005D0410F4942D852D9B878C874D855E85C7
:102750006F857889E12C85019E01255F3F4FC3017C
:102760000E944712182F882309F447C060E870E0E0
:102770008BE894E00E94081D60E870E0812F0E94C1
:10278000C30860E870E088E894E00E94081D1630F5
:1027900009F070C060E870E084E894E00E94081DD1
:1027A000C8CF80E894E00E94081D6F857889FB01FE
:1027B0008281816082834D855E8585019201C3019E
:1027C0000E946011182F882309F456C060E870E059
:1027D00089E794E00E94081D60E870E0812F0E9464
:1027E000C30860E870E086E794E08ACF111142C028
:1027F0002D853E85311024C041C0AAA5BBA5AB2BB9
:10280000A9F0AAA5BBA5ED91FC9111970190F081CB
:10281000E02DC4018C199D099A8789876B857C8579
:102820009E01275F3F4FA501CD0109958B859C85B2
:10283000C81AD90A8415950508F07BCF2D853E85E9
:1028400060EA4F2DC3010E943E10182F882381F0AB
:1028500060E870E080E794E00E94081D60E870E0A6
:10286000812F0E94C30860E870E08DE694E048CFB5
:1028700080E006C0812F04C02D853E8560E8E1CF51
:1028800061960FB6F894DEBF0FBECDBFDF91CF913A
:102890001F910F91FF90EF90DF90CF90BF90AF907E
:1028A0009F908F907F906F905F904F903F902F9070
:1028B00008958F929F92AF92BF92CF92EF920F9313
:1028C0001F931F921F921F930F933F932F934901C2
:1028D000A12CB12CCC24C394E12C06E020E80E946A
:1028E00014130F900F900F900F900F900F901F9157
:1028F0000F91EF90CF90BF90AF909F908F900895E1
:102900008F929F92AF92BF92CF92EF92FF920F93CE
:102910001F921F92FF92EF923F932F934901A12C98
:10292000B12C22E0C22EE02E06E020E80E94141313
:102930000F900F900F900F900F900F900F91FF90AE
:10294000EF90CF90BF90AF909F908F9008954F924F
:102950005F926F927F928F929F92AF92BF92CF922F
:10296000DF92EF92FF920F931F93CF93DF93CDB738
:10297000DEB7C054D1090FB6F894DEBF0FBECDBF8D
:102980003C01D62E542E422EC02ECE0101965C0163
:102990007C01022F29E030E0C3010E9480148111E4
:1029A0001BC08B809C801F93CF92BF92AF921F92CF
:1029B00080E48F93A12CB12C82E0C82EE42C06E099
:1029C00020E8452D6D2DC3010E9414130F900F9028
:1029D0000F900F900F900F90C05CDF4F0FB6F894E0
:1029E000DEBF0FBECDBFDF91CF911F910F91FF9042
:1029F000EF90DF90CF90BF90AF909F908F907F909F
:102A00006F905F904F9008958F929F92AF92BF9278
:102A1000CF92EF920F93CF931F921F921F921F920C
:102A20001F921F92812C912CA12CB12CC12CE22E33
:102A300005E020E00E941413C82F6CE271E080E0F2
:102A400090E00E947D0D0F900F900F900F900F90CF
:102A50000F908C2FCF910F91EF90CF90BF90AF90B0
:102A60009F908F9008950F931F93CF93DF938A3F8A
:102A70003FEF930711F486ED2DC0DC011696ED9122
:102A8000FC911797EF2B09F1122F242FEC011A87D5
:102A900040E00E94210E082F8823C9F0682FCE0144
:102AA0000E947A0E009739F3FC011483202F40E036
:102AB00060E0CE010E940415182F882351F0602F8A
:102AC000CE010E94DA0E812F05C087ED03C084ED90
:102AD00001C080E0DF91CF911F910F9108952F9257
:102AE0003F924F925F926F927F928F929F92AF929E
:102AF000BF92CF92DF92EF92FF920F931F93CF93EB
:102B0000DF93CDB7DEB766970FB6F894DEBF0FBE82
:102B1000CDBF1B8A38E03C8B3CE33D8B8A3F3FEFC7
:102B2000930709F464C0522E342E462E7C01DC013A
:102B30001696CD90DC901797CE01439617969C93EE
:102B40008E9316971A962C938E010F5F1F4F22E1DA
:102B500030E040E060E0C7010E945914F701D782DD
:102B6000C6828111A6C089849A846B847C84FD818D
:102B7000FE8B2E80670136E5C30ED11C560110E096
:102B8000D5018D919C910097F1F1DC01ED91FC91C3
:102B90000084F185E02D0995811135C0F501808112
:102BA0009181DC01ED91FC910088F189E02D622D8D
:102BB0000995882341F1F50180819181DC01ED9136
:102BC000FC910484F585E02DA301B40109958111E0
:102BD00010C0F50180819181DC01ED91FC910684AA
:102BE000F785E02D6E890995811103C00CC086ED33
:102BF00060C0052D232D442D612FC7010E94A11017
:102C0000813D09F056C01F5FB2E0AB0EB11C103120
:102C100009F0B6CF10E0F601808191810097E1F1D3
:102C2000DC01ED91FC910084F185E02D0995811185
:102C300033C0F60180819181DC01ED91FC91008827
:102C4000F189E02D622D09958823D9F0F601808164
:102C50009181DC01ED91FC910484F585E02DA301C7
:102C6000B4010995811118C0F60180819181DC01C0
:102C7000ED91FC910684F785E02D6E89099581110F
:102C80000BC0052D232D442D612FC7010E94A110DB
:102C9000982F977F913D69F41F5FE2E0CE0ED11C23
:102CA000103109F0B8CF252D432D642DC7010E94A6
:102CB000331566960FB6F894DEBF0FBECDBFDF9119
:102CC000CF911F910F91FF90EF90DF90CF90BF9029
:102CD000AF909F908F907F906F905F904F903F90BC
:102CE0002F9008958F929F92AF92BF92CF92EF92C2
:102CF0000F931F921F921F921F921F921F92812C5F
:102D0000912CA12CB12CC12CE22E09E020E00E94D4
:102D100014130F900F900F900F900F900F900F9132
:102D2000EF90CF90BF90AF909F908F9008957F923B
:102D30008F929F92AF92BF92CF92DF92EF92FF92CB
:102D40000F931F93CF93DF9300D000D0CDB7DEB7A2
:102D50006C01762EF42E590148011C821B821A82C6
:102D600019828E010F5F1F4F9E012D5F3F4F0E9402
:102D7000D10F182F8823A9F161E870E088E494E06E
:102D80000E94081D61E870E0812F0E94C30861E87D
:102D900070E085E494E00E94081D61E870E083E241
:102DA00094E00E94081D61E870E0872D0E94C3082E
:102DB00061E870E080E294E00E94081D61E870E044
:102DC00080E094E00E94081D61E870E08F2D0E9471
:102DD000C30861E870E08DEF93E00E94081D812F29
:102DE00009C049815A816B817C8184019501C601AA
:102DF0000E9447120F900F900F900F90DF91CF918C
:102E00001F910F91FF90EF90DF90CF90BF90AF9008
:102E10009F908F907F900895AF92BF92CF92DF9254
:102E2000EF92FF920F931F93CF938C011D990EC0C9
:102E300088EC0E94AD0F85FF05C0C8010E941608EE
:102E400060E201C060E088EC0E94BE0F80919101B9
:102E5000813039F040F0823079F0833079F5C1E08B
:102E60000CC083E106C080912403807F803131F162
:102E700081E18093240322C0C0E080912403807FFD
:102E80008031E9F40E947B0DDC01CB0188539F4F18
:102E9000AF4FBF4F8093200390932103A093220351
:102EA000B093230380E28093240380ED0E94AD0F52
:102EB000682F6F7D80ED0E94BE0F01C0C0E07801D9
:102EC00086E5E80EF11C6801A6E7CA0ED11C570181
:102ED000F501819191915F01009739F0DC01ED914D
:102EE000FC910680F781E02D0995AC14BD0481F7B3
:102EF00080912403803409F447C050F4803221F1DA
:102F00008033A1F1813109F08EC0F60110820AC030
:102F1000813509F464C0803809F476C0803509F041
:102F200082C045C0D7018D919D917D01009739F0F8
:102F3000DC01ED91FC910480F581E02D0995EC1404
:102F4000FD0481F782E16DC00E947B0D009120039A
:102F5000109121032091220330912303DC01CB0146
:102F6000801B910BA20BB30BB7FD5DC080ED0E94DF
:102F7000AD0F682F606280ED0E94BE0F61E088EEA9
:102F80000E94BE0F80E44DC088EE0E94AD0F80FD10
:102F90004AC060E488EC0E94BE0F88ED0E94AD0F2D
:102FA000682F686088ED0E94BE0F80E53AC088EC0B
:102FB0000E94AD0F86FF37C081E5809324030E94F5
:102FC0007B0DDC01CB014496A11DB11D8093200334
:102FD00090932103A0932203B093230324C00E9463
:102FE0007B0DC0902003D0902103E0902203F0904D
:102FF0002303DC01CB018C199D09AE09BF09B7FD84
:1030000012C080E8809324032C2F40E060E0C801C8
:103010000E946F15882321F0823D29F080EA01C0CB
:1030200080E980932403CF911F910F91FF90EF903F
:10303000DF90CF90BF90AF9008958F929F92AF9204
:10304000BF92CF92EF920F93CF93DF93CDB7DEB7BE
:10305000C054D1090FB6F894DEBF0FBECDBF5F9349
:103060004F939E012F5F3F4F3F932F931F9220E47A
:103070002F9320E8822E912C5B0132E2C32EE12CAB
:1030800006E021E840E0FC016681848195810E9490
:1030900014130F900F900F900F900F900F90C05C33
:1030A000DF4F0FB6F894DEBF0FBECDBFDF91CF91DB
:1030B0000F91EF90CF90BF90AF909F908F90089519
:1030C0008F929F92AF92BF92CF92DF92EF92FF9238
:1030D0000F93A42EB12C1F921F92DF92CF92FF92DA
:1030E000EF924701C22EE02E09E021E2462FFC01BB
:1030F0006681848195810E9414130F900F900F9028
:103100000F900F900F900F91FF90EF90DF90CF9066
:10311000BF90AF909F908F9008958F929F92AF92A3
:10312000BF92CF92EF920F93A62EB12C1F921F92B7
:103130001F921F921F921F92812C912CC22EE42E5F
:103140000AE021E240E0FC016681848195810E94D1
:1031500014130F900F900F900F900F900F900F91EE
:10316000EF90CF90BF90AF909F908F9008958F92E7
:103170009F92AF92BF92CF92EF920F93A62EB12C57
:103180001F921F921F921F921F921F92812C912CAF
:10319000C12CE42E0BE021E240E0FC016681848139
:1031A00095810E9414130F900F900F900F900F9025
:1031B0000F900F91EF90CF90BF90AF909F908F9016
:1031C0000895FC018285089581E0693009F080E06E
:1031D0000895CF93DF93EC018A819B81DC01ED910F
:1031E000FC910480F581E02D6A8509958A858134FA
:1031F00039F4EA81FB81EA58FF4F80818B7F80831D
:103200001A861B861C861D861E861F86188A80E0ED
:10321000DF91CF9108958F929F92AF92BF92CF92FC
:10322000EF920F93A42EB12CB22A1F921F921F92DD
:103230001F921F921F92812C912CC12CE62E01E02F
:1032400023E240E0FC016285828193810E94141395
:103250000F900F900F900F900F900F900F91EF9095
:10326000CF90BF90AF909F908F9008958F929F9234
:10327000AF92BF92CF92EF920F93A62EB12C1F92D6
:103280001F923F932F935F934F934A01C12CE12CE0
:1032900000E023EA40E0FC016285828193810E9484
:1032A00014130F900F900F900F900F900F900F919D
:1032B000EF90CF90BF90AF909F908F9008958F9296
:1032C0009F92AF92BF92CF92EF920F93A42EB12C08
:1032D000B22A1F921F921F921F921F921F92812C3F
:1032E000912CC12CE62E03E023E240E0FC01628534
:1032F000828193810E9414130F900F900F900F9072
:103300000F900F900F91EF90CF90BF90AF909F9044
:103310008F9008952F923F924F925F926F927F927B
:103320008F929F92AF92BF92CF92DF92EF92FF92D5
:103330000F931F93CF93DF93CDB7DEB7E9970FB607
:10334000F894DEBF0FBECDBFDC011A96DC90D11021
:1033500017C1122FC42E69AF3C01FC01A280B380BB
:10336000D501ED91FC910190F081E02D60E0C50167
:1033700009957C01009709F406C1FC0180809180C9
:103380008114910409F402C11301F4E02F0E311CE1
:10339000DC0111963C922E9214961C93FE013196FC
:1033A0002F018F0128E030E040E060E0D301129669
:1033B0008D919C9113970E945914F70114828111E9
:1033C000EEC08D81893009F0E4C01981D501ED91FD
:1033D000FC910280F381E02D2C2D41E069ADC50107
:1033E0000995F3018287882309F4D6C098859583CF
:1033F000282F40E060E0828193810E940415C82E4E
:10340000882391F0D7018D929C92D501ED91FC918A
:103410000480F581E02DD3011A966C91C5010995C0
:10342000F3011286DC2CBFC0212F113208F020E2FC
:10343000D7018D929C9221110CC0910142E0F301C1
:103440006285828193810E944C0FF82E811190C079
:1034500011C030E0820140E0D3011A966C911A97B6
:1034600012968D919C9113970E945914F82E8111F8
:103470007FC0E3CF1F921F925F924F921F9288E00E
:103480008F9358E0852E912CA12CB12C69E2C62E89
:10349000E12C06E020EA40E0F3016285828193811D
:1034A0000E941413F82E0F900F900F900F900F9012
:1034B0000F9081115DC08B81D3011B968C931B975C
:1034C000720100E028E030E040E01A966C911A9713
:1034D00012968D919C9113970E948014F82E811161
:1034E00047C02B813C81720140E0F30162858281FB
:1034F00093810E948014F82E81113AC0298130E016
:10350000CE0181967C0140E0D3011A966C911A9706
:1035100012968D919C9113970E948014F82E811120
:1035200027C02E8140E0F3016285828193810E9451
:103530007216F82E81111CC011E0D3011B968C91DC
:10354000811740F020E0412F68E0C3010E945F191D
:103550001F5FF3CFD3011296ED91FC911397EA58B8
:10356000FF4F80818460808381E050968C931BC0E4
:1035700060E870E087EA94E00E94081DDF2C13C029
:1035800049EDD42E10C036EDD32E0DC027EDD22E2E
:103590000AC091EDD92E07C084EDD82E04C0F701E2
:1035A00091828082D82E8D2DE9960FB6F894DEBFD9
:1035B0000FBECDBFDF91CF911F910F91FF90EF9084
:1035C000DF90CF90BF90AF909F908F907F906F9043
:1035D0005F904F903F902F900895CF92DF92FF928F
:1035E0000F931F93CF93DF9300D000D0CDB7DEB7FA
:1035F0008C01F62E19821A821B821C8220E0462F33
:1036000061E10E940B1920E04F2D60E1C8010E948A
:103610000B1920E04F2D64E0C8010E945F1983E080
:10362000C82ED12C9E012F5F3F4F44E050E06F2DFC
:10363000C8010E9436198823F1F020E04F2D64E183
:10364000C8010E940B1920E04F2D60E1C8010E94C3
:103650000B1964E170E080E090E00E947D0D0F9016
:103660000F900F900F90DF91CF911F910F91FF90CE
:10367000DF90CF90089589819A81AB81BC819D7F35
:1036800083309140A041B105C1F264E670E080E072
:1036900090E00E947D0D81E0C81AD10819F6CDCFC7
:1036A000FC0184E791E091838083738362831286B7
:1036B00013861486158616861786108A148288E06B
:1036C00085839CE3968391E09783808784E081875C
:1036D00061157105B1F0DB01AA5ABF4F80E090E09F
:1036E0002D913D91232B49F48B96880F991FDB0177
:1036F000A80FB91FED93FC930895019680319105B1
:1037000079F70895EF92FF920F931F93CF938C0157
:10371000C62F7A01FA0180819181A281B381813023
:10372000F3E09F07F1E0AF07B105D1F060F4811538
:10373000E1E09E07AE07B10571F181309140A140F3
:10374000B10571F064C0833021E0920720E1A20747
:10375000B105E1F183309340A041B105B9F157C003
:1037600080912503811153C020E04C2F61E1C801F5
:103770000E940B1920E04C2F60E1C8010E940B1938
:1037800020E04C2F64E0C8010E945F1981E0809323
:10379000250381EB3DC020E0462F61E1C8010E9476
:1037A0000B1920E04C2F60E1C8010E940B19109208
:1037B0002503F80162856770C770660F660F660F94
:1037C0006C2B828193810E94690F21C020E04C2FD5
:1037D00064E1C8010E940B1920E04C2F60E1C80190
:1037E0000E940B1964E170E080E090E00E947D0D82
:1037F000F8016285F70121812695217067704C2FB1
:10380000F801828193810E946F151092250380E058
:10381000CF911F910F91FF90EF900895CF92DF927B
:10382000EF920F931F93CF93DF93CDB7DEB72E9711
:103830000FB6F894DEBF0FBECDBF6C0181E090E003
:103840009E878D87E12C8E010F5F1F4F9E01235FA6
:103850003F4F41E0F6016285828193810E94971675
:10386000811151C002E011E089818023D1F01986D5
:103870001A861B861C869E01275F3F4F44E050E05E
:10388000612FC6010E94361981110BC0AE01475F3E
:103890005F4F612FC6010E94821B813B99F181110C
:1038A00032C0000F1F5F1830F9F611E0F601838572
:1038B000811740F119861A861B861C869E01275F98
:1038C0003F4F44E050E0612FC6010E94361981113C
:1038D00017C089859A85877091708130914081F4F5
:1038E0008B859C8581609C878B87AE01475F5F4F8E
:1038F000612FC6010E94821B813B21F0811103C010
:103900001F5FD4CF80E02E960FB6F894DEBF0FBEB7
:10391000CDBFDF91CF911F910F91EF90DF90CF90AE
:1039200008950F931F93CF93DF93FC0120892111FA
:1039300002C080E020C0EC010E947B0D0C851D853B
:103940002E853F85DC01CB01801B910BA20BB30BB5
:10395000B7FDEFCFCE010E940E1C182F0E947B0DE9
:10396000DC01CB018C599F4FAF4FBF4F8C879D8798
:10397000AE87BF87812FDF91CF911F910F9108955F
:10398000CF93DF93FC01EB0180819181892B39F585
:1039900060E870E081EB94E00E94081D24C0DA0129
:1039A0002D913C91232BF9F0A881B9819C91A381A1
:1039B000B0E0A81BB10920813181A20FB31F9C93F5
:1039C000828181508283DA018D919C9111970197B8
:1039D0008D939C93888199810196998388838281B4
:1039E0008111DDCF02C080E003C08381828381E04A
:1039F000DF91CF91089520910001309101012617A8
:103A000037072CF0682F8CEC92E00C94571D08952A
:103A10000F931F93CF93DF93209100013091010109
:103A20002617370774F0009761F08B01FC01849131
:103A3000EF012196882329F0B8010E94FB1CFE01AA
:103A4000F6CFDF91CF911F910F91089560E870E05C
:103A500089ED94E00C94081D60E870E08EEC94E031
:103A60000C94081DCF93C82F282F30E084E03595A3
:103A700027958A95E1F780E3820F8A3310F087E378
:103A8000820F60E870E00E94FB1CCF7080E38C0F17
:103A90008A3310F087E38C0F60E870E00E94FB1C13
:103AA00060E870E08BEC94E0CF910C94081DDC0191
:103AB000ED91FC910190F081E02D09948091320408
:103AC000089508950895CF93DF932091AC05243095
:103AD00049F521E02093E90021E8215059F0309187
:103AE000E80035FD07C0EFE3F1E03197F1F700C0E2
:103AF0000000F3CF2091E80025FF14C0EC0140E066
:103B000050E068E070E00E9437218091E8008E77F5
:103B10008093E80088E0FE01AAE2B4E001900D92F3
:103B20008A95E1F7DF91CF910895CF93C091280353
:103B3000C1110BC00E94E00D643C794081059105E4
:103B400020F081E080932803C1E08C2FCF9108956D
:103B5000FF920F931F93CF93DF93D82F0FB607FEDB
:103B600083C08091AC05843081F08091050190E0A4
:103B700001962091070130E08223932320910601D2
:103B800030E08217930709F0CDC00E94951D811186
:103B900010C08091050190E001962091070130E06E
:103BA000822393232091060130E08217930709F0C6
:103BB000B9C00E94D40D8C01C091E900CF709091E2
:103BC000EC00892F817090FD80E8C82B82E0809303
:103BD000E90085E0F82E8091EB0085FD42C08091E0
:103BE000EB0080FF3EC08091EE0087FF3AC08091DD
:103BF000060190910501981709F457C09091E800CB
:103C000095FF8EC0E0910301F0910401E80FF11DD2
:103C100020818F5F90910701892380930601209373
:103C2000F1008091E80085FDE2CF8091E80080FFFF
:103C3000DECF8091E8008E778093E800F092020159
:103C4000D6CF8091050190E001962091070130E0E8
:103C5000822393232091060130E08217930709F411
:103C60004CC0CF70C093E90040910501842F90E0D3
:103C700001962091070130E08223932320910601D1
:103C800030E08217930709F450C0E0910301F091EE
:103C90000401E40FF11DD083809105018F5F9091A5
:103CA000070189238093050140C08091E80085FFCA
:103CB00037C0D093F10021E03091F3008091F20001
:103CC00090E0932B892B91F08091E80080FF0EC04B
:103CD0008091E80085FF03C01092F100F9CF809138
:103CE000E8008E778093E800F0920201222309F425
:103CF000A8CFCF70C093E90018C08091020188233B
:103D000009F4AFCF0E94D40D9C018017910711F4E4
:103D1000890161CF90910201915090930201F8CFF7
:103D200020E0CACF40910501B0CF80E0DF91CF9174
:103D30001F910F91FF90089508958091AB05811117
:103D400004C00E94A3230C94002408951092AB0594
:103D50000895089542E061EC81E00E94B02042E2C3
:103D600061EC82E00C94B0208091AE05833009F4C0
:103D700053C030F4813071F0823009F48CC0089562
:103D80008A3009F478C08B3009F45EC0893009F0BC
:103D90009AC020C08091AD05813A09F094C080910D
:103DA000E800877F8093E8008091B1059091B2058B
:103DB000892B21F468E08AE294E003C060E080E0AF
:103DC00090E070E00E9484218091E8008B778093DE
:103DD000E80008958091AD05813209F074C08091AA
:103DE000B1059091B205892B09F06DC08091E80072
:103DF000877F8093E8008091E80082FD05C0809174
:103E0000AC058111F8CF5FC08091F100809332043E
:103E10008091E8008B7753C08091AD05813A09F01D
:103E200052C08091B1059091B205892B09F04BC029
:103E30008091E800877F8093E8008091E80080FF10
:103E4000FCCF8091120136C08091AD058132D9F549
:103E50008091B1059091B205892BA9F58091E80078
:103E6000877F8093E8000E94E5208091AF058093D2
:103E700012010C941F288091AD05813221F58091AB
:103E8000E800877F8093E8000E94E5208091B005DC
:103E90008093330408958091AD05813AA1F4809117
:103EA000E800877F8093E8008091E80080FFFCCFE6
:103EB000809133048093F1008091E8008E778093A5
:103EC000E8000C94E5200895809132048093290342
:103ED000109232040E947A260C941F280C94641FBE
:103EE0000E94D131809129038093320408950C946B
:103EF000701F08950C94791F0C94791FCF9384B789
:103F0000877F84BF0FB6F894A89580916000886180
:103F100080936000109260000FBE90E080E80FB6C2
:103F2000F89480936100909361000FBE88EA9DE150
:103F30000E94783188E091E00E9407258CE095E0AE
:103F40000E9497030E947C1F0E94BB250E94A3230E
:103F50000E94002478940E94BD258091AC05843095
:103F600029F00E94EC240E94791FF7CF8AEF94E099
:103F70000E9497030E947A1F88EE94E00E949703A4
:103F8000C2E08091AC05853019F40E94B207F9CFE8
:103F90000E94C1252091E4003091E5008091260324
:103FA000909127032817390709F468C08091E4002D
:103FB0009091E50090932703809326030E94951D1E
:103FC000882309F45BC08091AC05843009F056C0A9
:103FD0008091E9008F702091EC00922F917020FD6C
:103FE00090E8892BC093E9009091EB0090FF43C0CB
:103FF0009091EE0097FF3FC090910601209105013E
:10400000291709F12091E80025FF1DC0E091030167
:10401000F0910401E90FF11D30819F5F20910701AC
:104020009223909306013093F1009091E80095FD62
:10403000E3CF9091E80090FFDFCF9091E8009E776A
:104040009093E800D9CF9091F3002091F20030E0F6
:10405000392B232B81F09091E80090FF0CC09091B8
:10406000E80095FF03C01092F100F9CF9091E800AD
:104070009E779093E8008F708093E9000E94EC2473
:1040800080CF292F332723303105C9F060F4213048
:10409000310581F02230310509F044C082E490E01E
:1040A00025E735E043C021323105E1F02232310508
:1040B00049F138C082E190E027EB35E037C099271D
:1040C0008130910549F028F0029761F5E3E2F5E0CF
:1040D00005C0E1E7F5E002C0E1E6F5E0849190E09B
:1040E0009F0124C06115710541F061307105D1F463
:1040F00089E090E020EA35E019C089E090E027E807
:1041000035E014C06115710541F06130710551F45D
:1041100082E290E029EC35E009C080E490E02BEEEB
:1041200035E004C080E090E020E030E0FA01318327
:104130002083089580E189BD82E189BD09B400FE34
:10414000FDCF8091D8008F7D8093D8008091E000D2
:1041500082608093E0008091E00081FDFCCF0895B3
:10416000982F973068F59093E900981739F070917F
:10417000EC002091ED005091F00003C0242F762F29
:1041800050E021FD02C09F5FECCF3091EB003E7FFD
:104190003093EB003091ED003D7F3093ED00309196
:1041A000EB0031603093EB007093EC002093ED0056
:1041B0005093F0002091EE0027FDE5CF80E00895B8
:1041C0008F708093E90081E008958091AD0587FFAD
:1041D00011C08091E80082FD05C08091AC0581117D
:1041E000F8CF11C08091E8008B770BC08091AC05AF
:1041F000882349F08091E80080FFF8CF8091E800A3
:104200008E778093E80008952091E4003091E500D6
:1042100095E64091EC00842F817040FF23C080918F
:10422000E80080FD1DC08091AC05882399F08530A1
:1042300099F08091EB0085FD11C04091E400509110
:10424000E5002417350729F3915011F09A01E1CFC9
:1042500084E0089582E0089583E0089581E0089560
:1042600080E008954091E80042FFDDCF0895CF92AD
:10427000DF92EF92FF920F931F93CF93DF93EC01A6
:104280008B017A010E940421811135C0E114F104EF
:1042900039F0F70180819181081B190BC80FD91FD4
:1042A000C12CD12C0115110529F18091E80085FD63
:1042B00018C08091E8008E778093E8000E94EC247B
:1042C000E114F10449F0F70180819181C80ED91EF3
:1042D000D182C08285E00FC00E940421882311F39F
:1042E0000AC089918093F10001501109FFEFCF1AA4
:1042F000DF0AD8CF80E0DF91CF911F910F91FF901F
:10430000EF90DF90CF9008952091B3053091B405E0
:104310002617370748F06115710539F42091E80038
:104320002E772093E80001C0B901FC0120E061155F
:10433000710579F18091AC058823F1F18530F1F1B7
:104340008091E80083FD3CC08091E80082FD2EC092
:104350008091E80080FFEBCF2091F3008091F20084
:1043600090E0922B6115710551F08830910538F479
:1043700021912093F100615071090196F3CF21E062
:10438000089709F020E08091E8008E778093E8009C
:10439000CECF2111CFCF0AC08091AC05882361F028
:1043A000853061F08091E80083FD0AC08091E800CB
:1043B00082FFF2CF80E0089582E0089583E00895BF
:1043C00081E008952091B3053091B4052617370791
:1043D00048F06115710539F42091E8002E7720939B
:1043E000E80001C0B901FC0120E06115710591F1FF
:1043F0008091AC05882309F440C0853009F43FC0A2
:104400008091E80083FD3DC08091E80082FD2FC0CF
:104410008091E80080FFE9CF2091F3008091F200C5
:1044200090E0922B6115710559F08830910540F4A8
:1044300024912093F1003196615071090196F2CFD9
:1044400021E0089709F020E08091E8008E778093C2
:10445000E800CBCF2111CCCF0AC08091AC058823D6
:1044600061F0853061F08091E80083FD0AC08091A1
:10447000E80082FFF2CF80E0089582E0089583E0B3
:10448000089581E008951F93CF93DF93CDB7DEB7F2
:10449000AA970FB6F894DEBF0FBECDBFEDEAF5E0E8
:1044A0008091F100819325E0E53BF207C9F70E9476
:1044B000B41E8091E80083FF2EC18091AD059091DC
:1044C000AE05492F50E04A30510508F024C1FA01E9
:1044D000EA5AFF4F0C945E34803821F0823809F09C
:1044E0001AC108C08091A9059091AA05992389F065
:1044F00082600FC08091B1058F70873008F00BC1CA
:104500008093E9008091EB0085FB882780F9109269
:10451000E9009091E800977F9093E8008093F10084
:104520001092F100D1C0282F2D7F09F0F4C088230C
:1045300019F0823061F0EFC08091AF05813009F051
:10454000EAC0933009F080E08093AA052EC08091E4
:10455000AF0581112AC08091B1058F702FEF280F10
:10456000263008F0D8C08093E9002091EB0020FFAE
:104570001CC0933021F48091EB00806214C09091B4
:10458000EB0090619093EB0021E030E0A90102C0C4
:10459000440F551F8A95E2F74093EA001092EA0013
:1045A0008091EB0088608093EB001092E90080918D
:1045B000E800877F8093E8000E94E520ACC081116D
:1045C000AAC01091AF051F778091E3008078812BFE
:1045D0008093E3008091E800877F8093E8000E9449
:1045E000E5208091E80080FFFCCF8091E3008068A7
:1045F0008093E300111102C082E001C083E0809348
:10460000AC0589C08058823008F085C08091AF0524
:104610009091B0058C3D53E0950779F583E08A834E
:104620008AE289834FB7F894DE01139620E03EE0DA
:1046300051E2E32FF0E050935700E49120FF03C0D4
:10464000E295EF703F5FEF708E2F90E0EA3010F050
:10465000C79601C0C0968D939D932F5F243149F773
:104660004FBF8091E800877F8093E8006AE270E0A6
:10467000CE0101960E94842116C06091B10570910F
:10468000B205AE014F5F5F4F0E944120BC01892BF4
:1046900009F441C09091E800977F9093E8008981E8
:1046A0009A810E94E2218091E8008B778093E80054
:1046B00032C0803881F58091E800877F8093E800E0
:1046C0008091A8058093F1008091E8008E7772CFE9
:1046D000811121C08091AF059091B0059927029773
:1046E000D4F48091E800877F8093E8008091AF0543
:1046F0008093A8050E94E5208091A805811106C03D
:104700008091E30087FD02C081E001C084E08093D6
:10471000AC050E94AA1E8091E80083FF0AC0809128
:10472000E800877F8093E8008091EB0080628093AF
:10473000EB00AA960FB6F894DEBF0FBECDBFDF9197
:10474000CF911F9108950E9411240E941924E0EE38
:10475000F0E0808181608083E8EDF0E080818F77F8
:10476000808319BCA7EDB0E08C918E7F8C93808103
:104770008F7E80831092AB0508950F931F93CF9384
:10478000DF930E9411240E941924C8EDD0E0888193
:104790008F77888388818068888388818F7D8883EC
:1047A00019BC1092AC051092A8051092AA0510929F
:1047B000A90500EE10E0F80180818B7F808388815D
:1047C0008160888342E060E080E00E94B020E1EEFA
:1047D000F0E080818E7F8083E2EEF0E08081816076
:1047E0008083808188608083F80180818E7F8083D0
:1047F000888180618883DF91CF911F910F91089507
:10480000E8EDF0E080818F7E8083E7EDF0E080814D
:104810008160808384E082BF81E08093AB050C944B
:10482000BD23E8EDF0E080818E7F80831092E2006E
:1048300008951092DA001092E10008951F920F92ED
:104840000FB60F9211242F933F934F935F936F9363
:104850007F938F939F93AF93BF93EF93FF93809139
:10486000E10082FF0BC08091E20082FF07C08091CF
:10487000E1008B7F8093E1000E94EB248091DA00BD
:1048800080FF1FC08091D80080FF1BC08091DA009C
:104890008E7F8093DA008091D90080FF0DC080E187
:1048A00089BD82E189BD09B400FEFDCF81E080931E
:1048B000AC050E949D1E05C019BC1092AC050E945B
:1048C000A61E8091E10080FF19C08091E20080FF68
:1048D00015C08091E2008E7F8093E2008091E2001B
:1048E00080618093E2008091D80080628093D8003C
:1048F00019BC85E08093AC050E946E1F8091E10099
:1049000084FF30C08091E20084FF2CC080E189BD2B
:1049100082E189BD09B400FEFDCF8091D8008F7D72
:104920008093D8008091E1008F7E8093E100809198
:10493000E2008F7E8093E2008091E20081608093AC
:10494000E2008091A805882311F084E007C08091DF
:10495000E30087FD02C081E001C083E08093AC05E5
:104960000E94771F8091E10083FF24C08091E200C4
:1049700083FF20C08091E100877F8093E10082E087
:104980008093AC051092A8058091E1008E7F809302
:10499000E1008091E2008E7F8093E2008091E2004E
:1049A00080618093E20042E060E080E00E94B020FD
:1049B0000E94A91EFF91EF91BF91AF919F918F919E
:1049C0007F916F915F914F913F912F910F900FBE0B
:1049D0000F901F9018950895CF938091AC05882370
:1049E000A1F0C091E900CF709091EC00892F817007
:1049F00090FD80E8C82B1092E9008091E80083FDCB
:104A00000E944322CF70C093E900CF910895909304
:104A10003904809338040895E0913804F091390402
:104A2000309721F00190F081E02D099480E0089505
:104A3000EF92FF920F931F93CF93DF93E09138048F
:104A4000F09139043097B1F18C010280F381E02DAF
:104A500009958091A60582FF2DC080FF04C081E5E5
:104A600096E00E949703E80118E08BE4E82E86E0C8
:104A7000F82E8091A60580FF0BC088811F928F932E
:104A8000FF92EF920E9430040F900F900F900F90C2
:104A9000115021961111EDCF8091A60580FF0AC01B
:104AA00089E496E0DF91CF911F910F91FF90EF90F5
:104AB0000C949703DF91CF911F910F91FF90EF908E
:104AC0000895CF93DF93209136043091370428174F
:104AD000390709F19093370480933604E091380444
:104AE000F09139043097B9F0EC010680F781E02DA0
:104AF00009958091A60582FF0EC080FF0CC0DF9350
:104B0000CF938BE396E09F938F930E9430040F9096
:104B10000F900F900F90DF91CF910895CF93DF9377
:104B200020913404309135042817390709F1909306
:104B3000350480933404E0913804F09139043097BF
:104B4000B9F0EC010084F185E02D09958091A6056E
:104B500082FF0EC080FF0CC0DF93CF938BE296E004
:104B60009F938F930E9430040F900F900F900F909F
:104B7000DF91CF9108950C947B260E94CB0D0C946D
:104B8000A1088F929F92AF92BF92CF92DF92EF9245
:104B9000FF920F931F93CF93DF9300D000D01F920B
:104BA000CDB7DEB70E9440060BE314E0F12C8F2D49
:104BB0000E9428074C01F801A080B180A826B926E0
:104BC000A114B10439F4F3940E5F1F4FF0E1FF120A
:104BD000EECF39C08091A60581FD0E945507E12CDA
:104BE000CC24C394D12CC5018C219D21892B21F18A
:104BF000E982FA8221E0C4018C219D21892B09F4EC
:104C000020E02B830E94D40D8160782F9D838C83BC
:104C100049815A816B818D810E947E2649815A810A
:104C20006B817C818D810E947E31F8018081918130
:104C30008C259D2591838083E394CC0CDD1CF0E1D1
:104C4000EF12D1CFC0CF8FEF89838A831B820E945E
:104C5000D40D8160782F9D838C8349815A816B812B
:104C60008D810E947E260E947D310E940C259091AC
:104C70003A04891759F10E940C2580933A049091C7
:104C8000A60592FF0EC090FF0CC01F928F938CE57B
:104C900096E09F938F930E9430040F900F900F9097
:104CA0000F9080913A040F900F900F900F900F90FB
:104CB000DF91CF911F910F91FF90EF90DF90CF90F8
:104CC000BF90AF909F908F900C948F310F900F906A
:104CD0000F900F900F90DF91CF911F910F91FF9048
:104CE000EF90DF90CF90BF90AF909F908F900895FE
:104CF0000C9456070895089508950895CF93DF936F
:104D0000CDB7DEB72B970FB6F894DEBF0FBECDBF81
:104D1000942F4F83252F588769877A878B874A85F9
:104D20005B85452B31F02F3F31F481E09F3F19F433
:104D300003C081E001C080E080FD07C04F8158853D
:104D400069857A858B850E947E31DE01119686E029
:104D5000FD0111928A95E9F785E0FE0137960190F1
:104D60000D928A95E1F749815A816B817C818D8111
:104D70009E810E94FC2D2B960FB6F894DEBF0FBECD
:104D8000CDBFDF91CF910895CF93DF93882309F4AE
:104D9000E8C09EE7980F933018F5823829F08338E1
:104DA00031F0C4E0D7E405C0C2E0D9E302C0C1E0FD
:104DB000D3E50E940C258C2309F0D3C08D2F0E94CF
:104DC000DA300E9452312FEF81EE94E02150804082
:104DD0009040E1F700C000008D2F0E94F73006C020
:104DE0009CEF980F913A30F40E94DA30DF91CF9126
:104DF0000C94523190E2980F983050F4877091E003
:104E000001C0990F8A95EAF7892F0E941831EECFD9
:104E10009BE5980F933080F4853A29F0863A31F07B
:104E200083E890E005C081E890E002C082E890E06D
:104E3000DF91CF910C94612598E5980F973108F098
:104E400090C0883A09F445C0893A09F445C08A3AC5
:104E500009F445C08B3A09F445C08C3A09F445C0C1
:104E60008D3A09F445C08E3A09F445C08F3A09F4E9
:104E700045C0813B09F445C0803B09F445C0823BF5
:104E800009F445C0833B09F445C0843B09F445C09F
:104E9000853B09F445C0863B09F445C0873B09F4CE
:104EA00045C0883B09F445C0893B09F445C08A3BAD
:104EB00009F445C08B3B09F445C08C3B09F445C05F
:104EC0008D3B09F445C08E3B09F445C080E090E07D
:104ED00044C082EE90E041C089EE90E03EC08AEE90
:104EE00090E03BC085EB90E038C086EB90E035C0A9
:104EF00083EB90E032C084EB90E02FC087EB90E032
:104F00002CC08CEC90E029C08DEC90E026C083E8AA
:104F100091E023C08AE891E020C082E991E01DC0C1
:104F200084E991E01AC081E292E017C083E292E046
:104F300014C084E292E011C085E292E00EC086E2E5
:104F400092E00BC087E292E008C08AE292E005C0DE
:104F50008FE690E002C080E790E0DF91CF910C9463
:104F60008E25DF91CF910895CF93DF93882309F4A5
:104F70004FC09EE7980F933000F5823829F08338B0
:104F800031F0C4E0D7E405C0C2E0D9E302C0C1E01B
:104F9000D3E50E940C258C23D9F18D2F0E94DA30A5
:104FA0000E9452312FEF81EE94E0215080409040DA
:104FB000E1F700C000008D2F04C09CEF980F913ADC
:104FC00018F40E94F7300DC090E2980F983068F402
:104FD000877091E001C0990F8A95EAF7892F0E94A6
:104FE0001E31DF91CF910C9452319BE5980F933095
:104FF00030F480E090E0DF91CF910C946125885AE5
:10500000873130F480E090E0DF91CF910C948E25D1
:10501000DF91CF910895882321F00E9418310C94DC
:1050200052310895882321F00E941E310C94523190
:1050300008950E9438310E9407310C9452310E9429
:1050400028310C941928CF92DF92EF92FF920F93A0
:105050001F93CF93DF9300D000D01F92CDB7DEB760
:105060006C010E9491318111CDC285E0F601DE0113
:10507000119601900D928A95E1F7F60140815181D8
:10508000238134812115310531F05F3F31F481E016
:105090004F3F19F403C081E001C080E080FDB2C23F
:1050A000F601F280E580E2948FE0E82249835A839A
:1050B000FB82722F3D832C836F2D8D810E94563091
:1050C0008C010E9455300E944F2FE12FE295EF7026
:1050D0008E2F90E0FC01E05AFF4F0C945E34812F3C
:1050E000807F1F70882311F01295107FFF20B9F088
:1050F000112329F0812F0E942B310E945231802FE1
:105100000F900F900F900F900F90DF91CF911F9104
:105110000F91FF90EF90DF90CF900C94C426802FDA
:105120000E94B427112309F46DC2812F0E943131EE
:105130000F900F900F900F900F90DF91CF911F91D4
:105140000F91FF90EF90DF90CF900C945231812F10
:10515000807F1F70803211F01295107F002319F0AC
:10516000013009F12BC0FF20A9F0EE2059F1F1E048
:10517000812FEF1228C00F900F900F900F900F907B
:10518000DF91CF911F910F91FF90EF90DF90CF9023
:105190000C943B31EE2021F021E0E21609F432C2FA
:1051A0000E943E314DC0FF20E9F085E08E1508F4E5
:1051B00029C20E941531812329F042C0FF20F1F15C
:1051C000E11015C0812F0F900F900F900F900F904E
:1051D000DF91CF911F910F91FF90EF90DF90CF90D3
:1051E0000C940B2894E09E1508F40CC229C0F6011B
:1051F000858180FF13C08F708583E4CF003F09F461
:105200003EC108F00AC180E4800F803208F40EC16C
:10521000FF2009F49FC1EE2009F44FC1802F0E94A6
:10522000C426093309F08FC1FFEF21EE84E0F1506D
:1052300020408040E1F700C00000E4C1E1108CC1D3
:10524000812F0EC1812F837009F070C0F110DAC177
:10525000202F229526952770220F220F602F6F7026
:10526000862F90E0A0E0B0E06C017D01022E04C02A
:10527000CC0CDD1CEE1CFF1C0A94D2F704FF12C0FC
:105280008FE090E0A0E0B0E004C0880F991FAA1F53
:10529000BB1F2A95D2F7BC01CD0160957095809512
:1052A000909503C060E070E0CB01169516951370E1
:1052B0001230B1F040F56C297D298E299F291130DB
:1052C00031F10F900F900F900F900F90DF91CF91D1
:1052D0001F910F91FF90EF90DF90CF900C946A2F69
:1052E0006C297D298E299F290F900F900F900F9088
:1052F0000F90DF91CF911F910F91FF90EF90DF9072
:10530000CF900C94842F0E946A2FC701B6010F9092
:105310000F900F900F900F90DF91CF911F910F91F1
:10532000FF90EF90DF90CF900C94502FFF2019F05A
:10533000812F817001C08695882309F463C1202FD5
:10534000229526952770220F220F602F6F70862FCF
:1053500090E0A0E0B0E06C017D01022E04C0CC0C16
:10536000DD1CEE1CFF1C0A94D2F704FF12C08FE074
:1053700090E0A0E0B0E004C0880F991FAA1FBB1FF7
:105380002A95D2F7BC01CD016095709580959095D6
:1053900003C060E070E0CB011695169513701230D3
:1053A000B1F040F56C297D298E299F29113031F10A
:1053B0000F900F900F900F900F90DF91CF911F9152
:1053C0000F91FF90EF90DF90CF900C9431306C29CB
:1053D0007D298E299F290F900F900F900F900F908D
:1053E000DF91CF911F910F91FF90EF90DF90CF90C1
:1053F0000C9443300E943130C701B6010F900F90DA
:105400000F900F900F90DF91CF911F910F91FF9010
:10541000EF90DF90CF900C941F30023F09F45EC0F4
:1054200008F449C0033F09F46CC0F2CE902F90718C
:10543000E92E812F8F71FF2051F00E94B82F802F0D
:10544000EE2019F08295807FBECE8F70BCCE0E9478
:10545000D92F802FEE2019F08295807F01C08F70A8
:105460000F900F900F900F900F90DF91CF911F91A1
:105470000F91FF90EF90DF90CF900C941228FF20B7
:10548000A9F0E4E0EE1508F4BDC0812F8F710F90F4
:105490000F900F900F900F90DF91CF911F910F9170
:1054A000FF90EF90DF90CF900C94FE2FF5E0FE156B
:1054B00008F4A8C0EACFFF2099F0812F8F710F90D8
:1054C0000F900F900F900F90DF91CF911F910F9140
:1054D000FF90EF90DF90CF900C94B82FFF2069F3EE
:1054E000812F8F710F900F900F900F900F90DF9181
:1054F000CF911F910F91FF90EF90DF90CF900C9480
:10550000D92FFF2089F0812F8F710F900F900F906E
:105510000F900F90DF91CF911F910F91FF90EF901F
:10552000DF90CF900C94A32F0F900F900F900F90BF
:105530000F90DF91CF911F910F91FF90EF90DF902F
:10554000CF900C949E2F033509F46ECE073409F0EA
:1055500059C06ACEEE2021F2802F0F900F900F904D
:105560000F900F90DF91CF911F910F91FF90EF90CF
:10557000DF90CF900C94B427412F4F70602FC6015D
:105580000E941D320F900F900F900F900F90DF919F
:10559000CF911F910F91FF90EF90DF90CF900C94DF
:1055A000AA2E01112FC0FF2069F10E941F282FEFA2
:1055B00080E792E0215080409040E1F700C0000079
:1055C0000F900F900F900F900F90DF91CF911F9140
:1055D0000F91FF90EF90DF90CF900C94FE31412F10
:1055E0004F70602FC6010F900F900F900F900F908B
:1055F000DF91CF911F910F91FF90EF90DF90CF90AF
:105600000C9420320F900F900F900F900F90DF911D
:10561000CF911F910F91FF90EF90DF90CF90089561
:105620001F93CF93DF9300D000D01F92CDB7DEB78A
:10563000942F4983252F5A836B837C838D834C81E0
:105640005D81452B31F02F3F31F481E09F3F19F40C
:1056500003C081E001C080E0182F117080FD31C0CF
:1056600049815A816B817C818D810E945630292F1E
:1056700022952F702C3030F42A30A0F422502230A2
:1056800030F022C02C30C9F02F30B9F01DC0853A5F
:1056900028F48430C0F4823028F415C090E2980FCA
:1056A000983088F0883E30F4803E68F48450813A27
:1056B00058F409C0803F41F406C093FB112710F94C
:1056C00003C010E001C011E0812F0F900F900F90E8
:1056D0000F900F90DF91CF911F910895CF93DF939B
:1056E00000D000D01F92CDB7DEB70F900F900F9073
:1056F0000F900F90DF91CF910895CF93DF9300D05B
:1057000000D000D0CDB7DEB726960FB6F894DEBF36
:105710000FBECDBFDF91CF9108951F93CF93DF933D
:10572000C0915B0416E080915C04C81799F0D0E04A
:105730001C9FF0011D9FF00D1124E35AFB4F408187
:10574000518162817381848195810E947D2B219694
:10575000C770E9CFDF91CF911F91089540918D04DB
:1057600050918E0460918F04709190048091910407
:10577000909192040C947D2B0F931F93CF93DF9302
:105780008091920482958F7009F05DC080918F04A2
:10579000882309F458C080915B0410915C046091E7
:1057A0008D0470918E04C0919004D091910491E089
:1057B0006F3F09F090E0292F06E0811709F443C0FC
:1057C000209721F07F3F21F030E003C031E001C09D
:1057D000322F90E030FD34C0089FF001099FF00D9A
:1057E0001124DF01A35ABB4F11963C911197371337
:1057F00027C03C91361324C012963C911297311168
:105800001FC013964D915C9114974C1B5D0B483C47
:105810005105B0F4809192048F708061809392045E
:10582000EE59FB4F80818F70806180838DE894E01A
:105830000E942328DF91CF911F910F910C948D2B03
:1058400001968770BACFDF91CF911F910F91089584
:105850009F92AF92BF92CF92DF92EF92FF920F93FF
:105860001F93CF93DF93CDB7DEB761970FB6F89450
:10587000DEBF0FBECDBF8C0185E0F801DE011D96B5
:1058800001900D928A95E1F7F80140815181F280F3
:10589000C380D48090918D0460918E0420919004F7
:1058A000309191042115310531F06F3F31F481E0E1
:1058B0009F3F19F403C081E001C080E0F82FF17030
:1058C0009F2E80FD52C18DE8A82E84E0B82EE09076
:1058D0008F04F601E21BF30BEE2009F4E8C080917F
:1058E0009204E83CF10508F0A4C0282F207F09F0BD
:1058F00053C0561313C0491311C0EF2CF1100EC042
:105900008F708061809392040E94AE2BC5010E942B
:10591000232880919204F80185835BC1C114D104CE
:1059200031F05F3F31F481E04F3F19F403C081E073
:1059300001C080E080FD03C081E08F2502C080E0CF
:1059400090E0F82FF170EF2E80FF1CC080915B0477
:1059500020915C0436E0821709F418C190E0389F6A
:10596000F001399FF00D1124E35AFB4F618156136A
:1059700006C06081461303C06281F61203C001961F
:105980008770E9CFEF2CFF2009F423C180919204A6
:1059900081608093920462C0561306C0491304C00C
:1059A000F11002C0F801A7C04D875E87FF867C2DED
:1059B000D98AC88A6F2D89890E94102B882399F172
:1059C000FF2089F120919204822F82958F7090E0C0
:1059D000029774F080918D0490918E0498878F8344
:1059E0001986DB86CA862C87CE0107960E9423285B
:1059F00086E0F801ADE8B4E001900D928A95E1F7F8
:105A00000E94BC2B0E94AE2B11C0561749F14D8746
:105A10005E87FF867C2DD98AC88A6F2D89890E946E
:105A2000102B81112CC0C8010E942328EE24E3947E
:105A3000D0C0282F207F49F77C2DD98AC88A6F2DA6
:105A400089890E946E2B8DE894E00E94232886E0CD
:105A5000F50111928A95E9F70E94AE2BE12CB9C0AD
:105A60004913D5CFF110D3CFF8018583C8010E9427
:105A7000232886E0F50111928A95E9F7AAC0FF2054
:105A800091F220919204822F82958F7090E002977C
:105A90000CF4AECF80918D0490918E049A8389830B
:105AA0001B82DD82CC822E83CE0101969FCFE83C03
:105AB000F10508F04BC0EF2CFF2009F4B4CF5613CA
:105AC00030C049132EC02091920420FD21C0822FA6
:105AD00082958F70482F50E041155105C9F0F801AB
:105AE00025834F30510541F08F5F982F9295907F1D
:105AF000822F8F70892B8583C8010E94232886E01E
:105B0000F801ADE8B4E001900D928A95E1F72AC062
:105B100086E0F801ADE8B4E001900D928A95E1F7D6
:105B200058C04D875E87FF867C2DD98AC88A6F2D25
:105B300089890E94102B81115BCF80919204816032
:105B400080939204C8010E94232843C07C2DD98AE7
:105B5000C88A6F2D89890E946E2B86E0F50111920B
:105B60008A95E9F70E94AE2B34C0FF2009F45BCF81
:105B70004D875E87FF867C2DD98AC88A6F2D8989DB
:105B80000E94102B882309F44ECF32CF7C2DD98A66
:105B9000C88A6F2D89890E945630292F22952F702F
:105BA000223028F49F7039F0811105C00BC02430D9
:105BB00028F49F7049F4805E883020F0C8010E946C
:105BC00023289E2CE92C05C0F8019581907F99F738
:105BD000F9CF8E2D61960FB6F894DEBF0FBECDBF04
:105BE000DF91CF911F910F91FF90EF90DF90CF90B9
:105BF000BF90AF909F9008951F93CF93DF93CDB741
:105C0000DEB72C970FB6F894DEBF0FBECDBF4F8323
:105C1000588769877A878B879C87CE0107960E9471
:105C2000282C8823D1F09F8188852A853B85232BCA
:105C300031F08F3F31F481E09F3F19F403C081E0E0
:105C400001C080E080FD47C04F81588569857A8515
:105C50008B859C850E947D2B3EC086E0FE01379699
:105C6000DE01119601900D928A95E1F7FF81E8859A
:105C70006A857B856115710531F0EF3F31F481E074
:105C8000FF3F19F403C081E001C080E080FD23C024
:105C900020915C0430E0C9010196877099274091FA
:105CA0005B0450E084179507F1F1F983EA837D8363
:105CB0006C8396E0929FD001939FB00D1124A35A5C
:105CC000BB4FFE01319601900D929A95E1F78093BA
:105CD0005C040E948D2B16E080915B0490915C0423
:105CE000891771F1189FC0011124835A9B4F0E949C
:105CF000282C882329F1E0915B041E9FF0011124D8
:105D0000E35AFB4F40815181628173818481958187
:105D10000E947D2B80915B0490E00196877099270B
:105D200080935B04D9CF0E941F2810925C041092CC
:105D30005B04EDE8F4E086E0DF011D928A95E9F767
:105D40002C960FB6F894DEBF0FBECDBFDF91CF917A
:105D50001F910895DF92EF92FF920F931F93CF93BD
:105D6000DF93FC01892B09F488C0E12CF12CDD24A0
:105D7000D394EF0121968491853709F460C058F4DB
:105D8000843708F04EC0843008F068C08130D1F00C
:105D9000823071F172C0883709F45BC050F48637E5
:105DA00009F453C0873709F068C08E2D0E94253151
:105DB00052C09CE7980F903708F05FC08F770E9421
:105DC000B4274EC08F010E5F1F4FFE01849190E2F9
:105DD000980F983050F48770FD2D01C0FF0F8A9501
:105DE000EAF78F2F0E942B3115C00E94C42614C0E1
:105DF0008F010E5F1F4FFE01849190E2980F983043
:105E000068F48770FD2D01C0FF0F8A95EAF78F2F88
:105E10000E9431310E945231E80122C00E94B42711
:105E2000FBCFCF010296FE01C491CC2361F0EFE9D4
:105E3000FFE03197F1F700C00000C150F6CFCF016D
:105E40000296FE01F490EC010BC00E941531E82E81
:105E500007C00E9428310E94523102C00E94C4260D
:105E60008F2D882341F0EFE9FFE03197F1F700C073
:105E700000008150F6CFFE017CCFDF91CF911F91C2
:105E80000F91FF90EF90DF900895609393057093CA
:105E9000940580939505909396050C948E31089502
:105EA0000F931F93009197051091980520919905E4
:105EB00030919A05602B712B822B932B6093970561
:105EC000709398058093990590939A051F910F916F
:105ED0000C948D310F931F930091970510919805A5
:105EE0002091990530919A05602371238223932391
:105EF00060939705709398058093990590939A0500
:105F00001F910F910C948D310F931F930091970562
:105F1000109198052091990530919A056027712775
:105F2000822793276093970570939805809399052E
:105F300090939A051F910F910C948D3160E070E061
:105F4000CB010C94452F0F931F9341E050E060E08C
:105F500070E08A019B0104C0000F111F221F331F34
:105F60008A95D2F7C901B8011F910F910C94452F62
:105F70000F931F9341E050E060E070E004C0440FD5
:105F8000551F661F771F8A95D2F7809193059091D0
:105F90009405A0919505B09196058A019B01082B67
:105FA000192B2A2B3B2BC901B8011F910F910C947F
:105FB000452F0F931F9341E050E060E070E004C074
:105FC000440F551F661F771F8A95D2F7409550954D
:105FD000609570958091930590919405A091950599
:105FE000B09196058A019B01082319232A233B239C
:105FF000C901B8011F910F910C94452F0F931F9366
:1060000041E050E060E070E004C0440F551F661F9F
:10601000771F8A95D2F78091930590919405A0916E
:106020009505B09196058A019B01082719272A2713
:106030003B27C901B8011F910F910C94452F0F9375
:106040001F9300919305109194052091950530912F
:106050009605602B712B822B932B1F910F910C9423
:10606000452F0F931F930091930510919405209154
:1060700095053091960560237123822393231F9108
:106080000F910C94452F0F931F930091930510913E
:1060900094052091950530919605602771278227F8
:1060A00093271F910F910C94452F08958F929F92E3
:1060B000AF92BF92DF92EF92FF920F931F93CF9315
:1060C000DF9300D000D01F92CDB7DEB76B837C8307
:1060D0008D838A018C819D81892B31F01F3F31F4A2
:1060E00081E04F3F19F403C081E001C080E080FFF0
:1060F00003C080E090E04DC08B818823D1F1809077
:10610000930590909405A0909505B0909605809188
:10611000970590919805A0919905B0919A05882AC4
:10612000992AAA2ABB2A8FE1E82EF12CD501C401B5
:106130000E2C04C0B695A795979587950A94D2F72B
:1061400080FD06C081E0E81AF10880F7D12C07C075
:10615000DE2CB8018E2D0E943C32019799F380E12C
:10616000189FF0011124ED56FB4FE00FF11DD08276
:1061700009C080E1189FF0011124ED56FB4FE00F9C
:10618000F11DD08009831A8369817A818D2D0E9447
:106190003C320F900F900F900F900F90DF91CF91A6
:1061A0001F910F91FF90EF90DF90BF90AF909F9065
:1061B0008F9008952091130130911401F9013296C6
:1061C0009FEF40E05191851789F09F3F19F45111DD
:1061D00001C0942F4F5F4630A9F79F3F39F0F90176
:1061E000E90FF11D97FDFA95828308950895E091D6
:1061F0001301F09114019F012A5F3F4F928189138F
:1062000001C012823196E217F307C1F7089581E0C9
:1062100090E0E0911301F0911401E80FF91F108252
:10622000019688309105A9F708958091A5050895F4
:106230009091A505892B8093A5050895809590914F
:10624000A50589238093A50508958093A505089544
:106250001092A50508959091A405892B8093A4051B
:10626000089580959091A40589238093A4050895AD
:106270001092A405089580939B05089510929B05A4
:1062800008958091130190911401FC0131969C01B5
:10629000285F3F4F80E0919191118F5FE217F307E4
:1062A000D1F70895E0911301F09114018091A505B3
:1062B0008083E0911301F091140190818091A405F5
:1062C000892B808380919B05882361F0E0911301E5
:1062D000F09114019081892B80830E9441318111BA
:1062E00010929B0580911301909114010C94182534
:1062F000909387018093860108950895CF93DF934B
:1063000000D000D01F92CDB7DEB70F900F900F9046
:106310000F900F90DF91CF910895089508950C94F8
:10632000782680E008958091AC05843021F11092A8
:10633000A70520E488E190E00FB6F894A895809333
:1063400060000FBE2093600083B7817F846083BFAD
:1063500083B7816083BF7894889583B78E7F83BF2E
:106360000FB6F894A89580916000886180936000D2
:10637000109260000FBE0895CF930E947C260E9469
:1063800040060E947D26C0E08C2F0E942807892BA2
:1063900029F4CF5FC031C1F780E001C081E0CF9127
:1063A00008950E947A260C941F281F920F920FB610
:1063B0000F9211248F939F93AF93BF938091A70562
:1063C000811113C080911C0390911D03A0911E03A5
:1063D000B0911F034196A11DB11D80931C039093A2
:1063E0001D03A0931E03B0931F03BF91AF919F9114
:1063F0008F910F900FBE0F901F9018950E94A323AE
:10640000F89487E797E7909301088093000887E066
:1064100090EBDC018093B5059093B605A093B7058A
:10642000B093B8059CE088E10FB6F894A8958093E6
:1064300060000FBE90936000FFCF80E090E0089571
:106440000895E72FF0E090E1899FE00DF11D112400
:1064500084E0EE0FFF1F8A95E1F7E60FF11DE05291
:10646000FF4F84910895E82FF0E0EE0FFF1FE05AF0
:10647000F0408591949108950E94213290E4980F04
:10648000903218F40E94333208958F3B50F4883ACA
:1064900048F5853AD0F48430A8F4813009F4B2C0CC
:1064A000AEC0883E40F4803E68F48F3B09F0A7C040
:1064B00020E030EEA9C0803F08F4A1C0282F30E0D2
:1064C0003065A2C0282F30E09FC0853A29F0863A77
:1064D00031F023E830E498C021E830E495C022E8A8
:1064E00030E492C0883A09F445C0893A09F445C0BD
:1064F0008A3A09F445C08B3A09F445C08C3A09F44C
:1065000045C08D3A09F445C08E3A09F445C08F3A2A
:1065100009F445C0813B09F445C0803B09F445C0FE
:10652000823B09F445C0833B09F445C0843B09F430
:1065300045C0853B09F445C0863B09F445C0873B0F
:1065400009F445C0883B09F445C0893B09F445C0BE
:106550008A3B09F445C08B3B09F445C08C3B09F4E8
:1065600045C08D3B09F445C08E3B09F445C020E091
:1065700034E44AC022EE34E447C029EE34E444C097
:106580002AEE34E441C025EB34E43EC026EB34E48B
:106590003BC023EB34E438C024EB34E435C027EBB4
:1065A00034E432C02CEC34E42FC02DEC34E42CC0A5
:1065B00023E835E429C02AE835E426C022E935E499
:1065C00023C024E935E420C021E236E41DC023E2E3
:1065D00036E41AC024E236E417C025E236E414C0DB
:1065E00026E236E411C027E236E40EC02AE236E4A1
:1065F0000BC02FE634E408C020E734E405C020E0F7
:1066000030E002C021E030E0C90108950E947733F4
:1066100008F481E008950E94CB3388F09F5798F0EA
:10662000B92F9927B751B0F0E1F0660F771F881F97
:10663000991F1AF0BA95C9F714C0B13091F00E94B1
:10664000E533B1E008950C94E533672F782F882760
:10665000B85F39F0B93FCCF3869577956795B395D8
:10666000D9F73EF490958095709561957F4F8F4F47
:106670009F4F0895E89409C097FB3EF4909580954C
:10668000709561957F4F8F4F9F4F9923A9F0F92FF8
:1066900096E9BB279395F695879577956795B79576
:1066A000F111F8CFFAF4BB0F11F460FF1BC06F5F5C
:1066B0007F4F8F4F9F4F16C0882311F096E911C06E
:1066C000772321F09EE8872F762F05C0662371F08F
:1066D00096E8862F70E060E02AF09A95660F771FA3
:1066E000881FDAF7880F9695879597F90895990F7F
:1066F0000008550FAA0BE0E8FEEF16161706E8078C
:10670000F907C0F012161306E407F50798F0621BAC
:10671000730B840B950B39F40A2661F0232B242B81
:10672000252B21F408950A2609F4A140A6958FEFA0
:10673000811D811D089597F99F6780E870E060E0F2
:1067400008959FEF80EC089500240A94161617060A
:1067500018060906089500240A9412161306140652
:1067600005060895092E0394000C11F4882352F0B5
:10677000BB0F40F4BF2B11F460FF04C06F5F7F4F6D
:106780008F4F9F4F089557FD9058440F551F59F054
:106790005F3F71F04795880F97FB991F61F09F3F0E
:1067A00079F087950895121613061406551FF2CF37
:1067B0004695F1DF08C0161617061806991FF1CF87
:1067C00086957105610508940895E894BB276627AE
:1067D0007727CB0197F908950E94773308F48FEF5C
:1067E00008950E9404340C94B2330E94A43338F00C
:1067F0000E94AB3320F0952311F00C949B330C9442
:10680000A13311240C94E6330E94C33370F3959F97
:10681000C1F3950F50E0551F629FF001729FBB2797
:10682000F00DB11D639FAA27F00DB11DAA1F649F33
:106830006627B00DA11D661F829F2227B00DA11DE6
:10684000621F739FB00DA11D621F839FA00D611D6C
:10685000221F749F3327A00D611D231F849F600D8D
:10686000211D822F762F6A2F11249F5750409AF0B6
:10687000F1F088234AF0EE0FFF1FBB1F661F771F42
:10688000881F91505040A9F79E3F510580F00C940D
:106890009B330C94E6335F3FE4F3983ED4F3869544
:1068A00077956795B795F795E7959F5FC1F7FE2BAD
:1068B000880F911D9695879597F90895EE0FFF1F04
:0C68C0000590F491E02D0994F894FFCFAE
:1068CC008000052A030000FF5E1D631D611D9C1ED8
:1068DC00621D019C0566756C6C006C6F7700000086
:1068EC000000FD0400000000FC0400000000E508AE
:1068FC00390489046B0BA4043B043C04A704AC04CA
:10690C00B1047D048604B904FEFF0000F20400000B
:10691C000000E90C00000000590D5F0D550D580DDD
:10692C004F0D520D520D000000007A0E210EDA0EA2
:10693C00000000008A193904E918911CE118ED1ABD
:06694C003C04E4183E04C7
:00000001FF
